:1080000000000120A111010011E4000011E40000B2
:1080100011E4000011E4000011E400000000000081
:1080200000000000000000000000000011E400005B
:1080300011E400000000000011E40000B985000018
:1080400011E4000011E4000011E4000011E400005C
:1080500011E4000011E4000011E4000011E400004C
:1080600011E4000011E4000011E4000011E400003C
:1080700011E4000011E4000011E4000011E400002C
:1080800011E4000011E4000011E4000011E400001C
:1080900011E4000011E4000011E4000011E400000C
:1080A00011E400008DCE000011E4000011E4000096
:1080B00011E4000011E4000011E4000011E40000EC
:1080C00011E4000011E4000011E4000011E40000DC
:1080D00011E4000011E4000011E4000005CD0000EF
:1080E00011E4000011E4000011E4000011E40000BC
:1080F00011E4000011E4000011E4000011E40000AC
:1081000011E4000011E4000011E4000011E400009B
:1081100011E40000B9F6000011E4000011E40000D1
:1081200011E4000011E4000011E4000011E400007B
:1081300011E4000011E4000011E4000011E400006B
:1081400011E4000011E400001D87000011E40000AC
:1081500011E4000011E4000011E4000011E400004B
:1081600011E4000051CD000011E4000011E4000012
:1081700011E4000011E4000011E4000011E400002B
:0881800011E4000011E400000D
:10840000FFFFFFFFFFFFFFFFFFFFFFFF7EF9FFFF03
:1084100010B5054C237833B9044B13B10448AFF3BE
:1084200000800123237010BD0086FF1F00000000A4
:108430005419010008B5064B1BB106480649AFF3B5
:1084400000800648036813B1054B03B1984708BD87
:1084500000000000541901000486FF1F6885FF1FFB
:108460000000000080F311887047304B41F2380261
:10847000995841F47851995041F23002995841F09D
:10848000807199502A4A927902F00C020C2A4CD041
:1084900041F244022749995003F558339A7812075C
:1084A00003D59A7842F008029A70204B224941F293
:1084B0004402995041F204015A5842F4803242F089
:1084C000C0025A501A6842F440221A6003F5E83399
:1084D00024225A70194A80211170A2221A70DA7867
:1084E00002F01F02DA7003221A7100225A719A797F
:1084F0009007FCD59A79D106FCD40D4B9A7902F0FD
:108500000C02082AF9D140225A719A7902F00C0221
:10851000082AFAD1064B9A795206FBD522221A7004
:108520009A7902F00C020C2AFAD1704700700440CC
:1085300000400640000033010000130100500640D7
:10854000184B5A7902F0E0025A711A7902F0F802D7
:108550001A71A3F55B33A3F570731A6842F0040235
:108560001A60114A136823F0784323F00103136063
:108570000E4B1A7802F08C0242F050021A705A78B0
:1085800002F09C0242F040025A709A7802F0E60231
:108590009A70074A00231370064A82F8353383F332
:1085A0001188704700F0074000D0004000D007401D
:1085B00000E0074000E100E0104B68461A6820F038
:1085C000070101328D4601B51A600D4B1A68013260
:1085D0001A600C4B1A683AB11A68013A1A601B68A3
:1085E00013B9094B01221A70084B1A6812B11A68A4
:1085F000013A1A60BDE80140854670471C86FF1F9E
:108600006498FF1FB093FF1FAC93FF1FB493FF1F2D
:10861000024B034A5A6007221A60704710E000E0DC
:1086200000770100014B1868704700BF1C86FF1FD0
:10863000072888BF0020134B134A53F8203010B589
:10864000124CB4FBF3F441F228034220D15841F418
:108650008061D1500E4B4FF440729A63DA6305F09B
:10866000EFFE0C4B0022DA709A709A71DA725A712E
:10867000C4F30422E4B21A705C70DA7842F02C027F
:10868000DA7010BD0817010000700440C0C62D004C
:1086900000B0044000A00E40094B1A68596801322E
:1086A000202A08BF00228A4208D01968194408729B
:1086B0001A60044BDA7842F08002DA70704700BF2B
:1086C0002086FF1F00A00E400A4B996ADA6A914289
:1086D0000CD09A6A511C1A44996292F830200270A8
:1086E0009A6A202A04D100229A6201E00020704791
:1086F000012070472086FF1F044B1A7802F0FF000C
:1087000012B100221A700120704700BFAC93FF1F06
:10871000014B1865704700BF2086FF1F684620F098
:1087200007018D4631B527480179C9B28C0615D5A8
:10873000254BDA6A9C6A0132202A08BF0022A24235
:1087400006D0DD6AC4795819E4B280F83040DA62A4
:108750001E4A052010601A6D1D4B1A604A0608D586
:108760001C4B4FF480529A60164BDA7802F0BF022D
:10877000DA700B0621D5164B1968F1B9124B18683F
:108780005A68904214D0134A4FF4805050605A688F
:10879000501C1A445860107A0A4AC0B2D071586806
:1087A000202808BF5960D37843F04003D37004E019
:1087B000044BDA7802F07F02DA70BDE8314085467A
:1087C000704700BF00A00E402086FF1FB093FF1F20
:1087D000B493FF1F80F00F4062B6704772B67047C7
:1087E00062B6704772B670474FF0E02308B1034A93
:1087F00000E0034AC3F80C2D704700BF0400FA05DF
:108800000100FA0513B53F4A3F484FF480730E212B
:108810004360836091605161A2F535224FF4F0010D
:1088200053629364D36413655365936502F53522EF
:10883000403251619160354A4FF490715162136337
:10884000936402F5342280324FF4905191604FF4DA
:108850008021516001F5905151612D4A40F2031180
:10886000116051609160D160116151619161D1617C
:1088700002F53322C03200245461264A264913618E
:1088800053619361936602F5322202F58072916022
:10889000516103600A21C360224623461948082417
:1088A000446000240194019CB4F57A7F02D2019CBB
:1088B0000134F7E70069C40712484FF008048460E8
:1088C00048BF013200240194019CB4F57A7F02D2A2
:1088D000019C0134F7E70069C00758BF0133013933
:1088E000DCD10A2A0D4A03D10A2B01D1012300E071
:1088F00000231370044B4FF4E0621A60DA6002B098
:1089000010BD00BF00F00F400090044000B00440D4
:1089100000C0044000D0044070000004EA93FF1F30
:10892000104B1B7882B0D3B10F4B02229A60042205
:108930005A600022019201990C4A914202D8019A90
:108940000132F7E702225A6004229A600023019361
:10895000019A064B9A42E7D8019B0133F7E702B030
:10896000704700BFEA93FF1F00F00F401FA10700F0
:1089700003280DD8DFE800F002040608102205E005
:10898000202203E0402201E04FF08062014B5A6058
:10899000704700BF00F10F4003280DD8DFE800F05A
:1089A00002040608102205E0202203E0402201E034
:1089B0004FF08062014B9A60704700BF00F10F409A
:1089C00038B50546002445FA04F3DB07E0B202D5CA
:1089D000FFF7CEFF01E0FFF7DFFF0134082CF2D1F3
:1089E00038BD08B5032813D8DFE800F002040608F4
:1089F000002004E0012002E0022000E0032004F057
:108A000015FA43F27C03984294BF0020012008BD70
:108A1000002008BD032817D8DFE800F002070C117A
:108A20000A4B1868C0F300107047084B1868C0F371
:108A300040107047054B1868C0F380107047034B17
:108A40001868C0F3806070470020704700F10F4045
:108A500038B500242546E0B2FFF7C3FF18B1012363
:108A6000A3401D43EDB20134082CF4D1284638BD93
:108A7000024B1869C043C0B2704700BFC0F00F403E
:108A800008B5082004F0D2F95E2804D9104B1A78F2
:108A90004AB9012206E0082004F0C8F9542802D897
:108AA0000B4B00221A70082004F0C0F9632804D987
:108AB000084B4FF400725A6008BD082004F0B6F964
:108AC000542803D8034B4FF400729A6008BD00BFCE
:108AD0007486FF1F80F00F40034B1878013801287F
:108AE0008CBF0020012070477486FF1F034B18784D
:108AF000012806BF02221A70002070477486FF1FEB
:108B0000C0B205F0B1B8C0B205F09CB80B4B10F084
:108B1000010F4FF4800214BF5A609A6010F0020FE8
:108B20004FF4001214BF5A609A6010F0040F4FF413
:108B3000801214BF5A609A60704700BF40F00F4027
:108B400008B507F0BDFB05F085FE05F035FEBDE874
:108B5000084007F037BC38B5054605F083FD082806
:108B60000AD900242819013405F0FCFD092CF9D19B
:108B700005F02CFE012038BD002038BD092105F08C
:108B800091BD002006F01AB8224A41F23C030120B0
:108B9000D15841F44051D1501F4B204918601A68F8
:108BA0000A431A601E4ADA601A61DA6A42F0805299
:108BB000DA621A6822F001021A601A6822F0006272
:108BC0001A60184A4FF40073136053609360D360C7
:108BD000136153619361D361A2F5F03210601068A4
:108BE000014311601049D16001F520011161D16A82
:108BF00041F08051D162116821F0010111601168CA
:108C000021F00061116002F5E8329362D3621364CF
:108C1000536470470070044000C00240000C1F8085
:108C20000300013E00B004400400513EFF2800F064
:108C30003F031AD82C4872B141F0006141EA034366
:108C40004363294BDA6A002A1946FADACA6A264BC4
:108C5000D200FBD541E041F0004141EA03434363C8
:108C6000214BDA6A002AFBDA37E0B0F5007F1AD22E
:108C70001E4872B141F0006141EA034343631B4B5C
:108C8000DA6A002A1946FADACA6A184BD000FBD50C
:108C900023E041F0004141EA03434363134BDA6AA6
:108CA000002AFBDA19E0124872B141F0006141EA92
:108CB000034343630E4BDA6A002A1946FADACA6A9A
:108CC0000B4BD200FBD508E041F0004141EA0343E1
:108CD0004363074BDA6A002AFBDA986BDA6A42F0E0
:108CE0001042C0B2DA62704700C0024000D00240B9
:108CF00000C00A4010B5FFF795FC0446FFF792FC50
:108D0000001B0028B8BF40420628F7DD10BD07B59C
:108D1000030A8DF805008DF80610032201A9A02092
:108D20008DF8043004F052F9FFF7E4FF03B05DF86A
:108D300004FB2DE9F04100238AB0884616461C4604
:108D4000B4421DD00AAA1A445D1C18F8041002F897
:108D5000221C2F18FA0602D0721E94420DD1020A6C
:108D60008DF804208DF8050001A9DA1CA02004F07C
:108D70002DF90025FFF7BEFF384601342B46DFE70B
:108D80000AB0BDE8F0811FB5030A022203A98DF8DD
:108D90000C308DF80D0000920B46A02004F06AF90B
:108DA0009DF80C0005B05DF804FB1FB50B46010AE9
:108DB0008DF80C108DF80D00009203A90222A0205E
:108DC00004F058F905B05DF804FBC0EBC00000F5F5
:108DD00000600722FFF7ADBFC0EBC00000F50060E8
:108DE0000722FFF7E2BF30B500238BB001AD0024AE
:108DF0005C550133222BF9D1230A8DF80540294611
:108E00002222A02020348DF8043004F0DFF8FFF790
:108E100071FFB4F5005FEFD10BB030BD13B50C4658
:108E2000C0EBC000072200F500606946FFF7BDFFF8
:108E30009DF8002023789A4211D19DF80120637893
:108E40009A420CD19DF80220A3789A4207D1DDF80E
:108E50000300D4F80330C31A5842584100E0002000
:108E600002B010BD704713B545F2FF70FFF78BFFDE
:108E7000AA2802D1254B1B78B3B345F2FF7000211D
:108E8000FFF745FFFFF7AFFF002021494022FFF722
:108E900050FF402420461F4940224034FFF749FF3D
:108EA000B4F5E07FF6D1002301934FF4D36420465C
:108EB00001A90422FFF73DFF043440F678039C42E9
:108EC000F5D1002301934FF4FF64204601A9042249
:108ED000FFF72FFF043440F6D8039C42F5D145F24A
:108EE000FF70AA21FFF713FF002009494022FFF776
:108EF0005CFF402408492046214440224034FFF7CB
:108F000054FFB4F5E07FF5D102B010BDEA93FF1F26
:108F10000C80FF1F38170100C093FF1FF7B5CE4E1E
:108F2000B4787278052C354600F26A84A32A00F0E2
:108F30005C8300F29880122A00F06C8242D8072AE3
:108F400000F0C3811AD8022A00F03B810CD8002A15
:108F500000F02881012A40F0558404F0010320210B
:108F6000994041F0010123E1052A00F07D8100F2E2
:108F70009581042A00F0498100F044BC0E2A00F0DB
:108F80000C8207D80C2A00F0C0810D2A00F0E18184
:108F900000F038BC102A4FEA540604F00107AF4B2A
:108FA00000F01F824FEA840400F228821C44D5F8A6
:108FB0000300236B9847202101FA07F7024647F088
:108FC000040119E2192A00F07C822DD8152A00F03C
:108FD0003E8213D8132A00F02C82142A40F0128407
:108FE0009E4BD6F8030053F82430984704F0010351
:108FF00020219940024641F00B0188E3172A4FEAED
:10900000540604F0010700F02D8200F23882934BE1
:10901000D5F8030053F824309847202101FA07F7C8
:10902000024647F01201E7E11F2A00F0A18210D8A2
:109030001B2A00F08E82C0F068821C2A40F0E28376
:10904000D6F803102046C9B203B0BDE8F04004F0E2
:10905000D6B98C2A00F0B582A22A00F0BD827F2A00
:1090600040F0D083A1E2B62A00F0448340D8AA2A77
:1090700000F0088318D8A62A00F0DD8206D8A42ABA
:1090800000F0BC82A52A00F0C282BBE3A82A00F04F
:10909000E78200F2EE82D6F803102046C9B203B090
:1090A000BDE8F04004F0DCB8AE2A00F006830DD82D
:1090B000AC2A00F0F08200F2F782D6F803102046C6
:1090C000C9B203B0BDE8F04004F021BBB32A00F000
:1090D000FD82B52A00F00383B12A40F09383D6F8CD
:1090E00003102046C9B203B0BDE8F04004F055B902
:1090F000C32A00F03B8323D8BB2A00F014830ED888
:10910000B82A00F00783B92A40F07C83D6F8031010
:109110002046C9B203B0BDE8F04004F00CB9C12A42
:1091200000F0138300F21883BC2A40F06B83D6F85A
:1091300003102046C9B203B0BDE8F04004F05CBCA7
:10914000D12A00F025831DD8CA2A00F01A83CC2A20
:1091500000F0F282C92A40F055836008182104F01B
:1091600027F800F48064B078202100F001029140DB
:10917000D6F8032041F0180122F480624008C9B2F9
:10918000224319E0D42A00F01183FF2A00F015834E
:10919000D22A40F03783324BD6F8032003EB8413F6
:1091A000DA61FDE204F001032021994041F00D0154
:1091B000D5F803206008C9B203B0BDE8F04003F061
:1091C000C7BFD6F803306008002B04F001044FF04D
:1091D000200303FA04F1C8BF0122C9B203F0B8FFAB
:1091E000B478204BD6F8030001221A551B4B0028F7
:1091F000B8BF404253F82430984704F001032021BF
:109200009940024641F0070181E2144ED5F803006F
:1092100056F824300028B8BF4042984706EB840433
:10922000A061A878202400F0010104FA01F14008AF
:10923000C9B203F0BDFF002840F0E782064B9878E2
:1092400000F0010106EB80068C4044F00701400865
:10925000C9B2B269B0E700BF5096FF1F7886FF1F02
:109260000094FF1FE293FF1FBE4BD6F803000022BD
:109270001A55BD4B03EB84031B6B9847B378BB4A6D
:1092800003F0010142F82400202000FA01F141F02E
:1092900006015808C9B252F823208DE7202604F0B1
:1092A000010106FA01F141F01001C9B2600803F0B2
:1092B0007FFF0346A878EA7800F00101D2088E40CB
:1092C000009246F01001DAB216E0202504F0010108
:1092D00005FA01F141F01001C9B2600803F068FF1E
:1092E0000346C3F30722B078009200F00101F27840
:1092F0008D4045F01001D20801924008C9B2002209
:10930000C3F3074303F0E8FE7FE204F001012026E7
:1093100006FA01F141F01401C9B2600803F048FFF8
:10932000D5F803100246A87849B900F001018E4033
:1093300046F014014008C9B242F002023CE700F0D6
:1093400001018E4046F014014008C9B222F0020229
:1093500032E704F00101202606FA01F141F0140180
:10936000C9B2600803F024FFD5F803100246A878BC
:1093700049B900F001018E4046F014014008C9B21D
:1093800042F0010218E700F001018E4046F014019E
:109390004008C9B222F001020EE704F001012025C5
:1093A00005FA01F141F01401C9B2600803F000FFB1
:1093B000D6F803100246B07849B100F001018D40A3
:1093C00045F014014008C9B242F01002F4E600F082
:1093D00001018D4045F014014008C9B222F010028D
:1093E000EAE653F82430D5F803009847202101FA23
:1093F00007F7024647F00501304689E11C44D5F8DD
:109400000300236B9847202101FA07F7024647F033
:109410000801F1E7544BD6F8030003EB84031B6B00
:10942000984704F0010320219940024641F00A01C7
:109430006DE14D4BD6F8030053F82430984704F003
:10944000010320219940024641F003015FE104F04D
:1094500001032021994041F00C016008C9B2D6F8FF
:109460000320A9E6404BD5F8030053F82430984771
:10947000202101FA07F7024647F01301BCE7202438
:1094800004FA07F747F01401C9B2304603F090FE22
:10949000D5F803100246A87849B100F001018C40CC
:1094A00044F014014008C9B242F0080284E600F01A
:1094B00001018C4044F014014008C9B222F00802B6
:1094C0007AE604F00101202505FA01F141F01401CA
:1094D000C9B2600803F06CFED6F803100246B078FB
:1094E00049B100F001018D4045F014014008C9B2B6
:1094F00042F0040260E600F001018D4045F01401E5
:109500004008C9B222F0040256E604F00101202608
:1095100006FA01F141F01401C9B2600803F048FEF7
:10952000D5F803100246A87849B100F001018E4039
:1095300046F014014008C9B242F400623CE600F073
:1095400001018E4046F014014008C9B222F40062C5
:1095500032E6D6F803102046C9B203B0BDE8F040A9
:1095600003F034BF4896FF1F7886FF1F3096FF1F19
:1095700004F00101202505FA01F141F01001600815
:10958000C9B203F015FEB278F37802F001018D4004
:10959000C0F3072445F01001C0B2019000945008B8
:1095A000C9B2002203F00F03ACE6D6F80330022B59
:1095B00000F22681964B1C44964BDB7884F84830A9
:1095C00023E1D6F80310C1F108012046C9B203B067
:1095D000BDE8F04003F0C8BED6F803102046C9B27B
:1095E00003B0BDE8F04003F08DBED6F8031020466E
:1095F000C9B203B0BDE8F04003F01ABFD6F80310BB
:109600002046C9B203B0BDE8F04003F043BF204696
:1096100004F02AF8D6F8031030B9B078C9B203B014
:10962000BDE8F04003F055BEB078C9B203B0BDE864
:10963000F04003F048BF204604F016F8B378D6F89F
:10964000031030B91846C9B203B0BDE8F04003F0CA
:1096500027BE1846C9B203B0BDE8F04003F053BFBF
:10966000D6F803102046C9B203B0BDE8F04004F0BC
:10967000C8B8D6F803102046C9B203B0BDE8F04020
:1096800004F05EB8D6F803102046C9B203B0BDE8B6
:10969000F04004F06EB8D6F803102046C9B203B00B
:1096A000BDE8F04004F07EB8D6F803102046C9B2F9
:1096B00003B0BDE8F04004F0BDB8D6F80310204672
:1096C000C9B203B0BDE8F04004F084B8D6F8031086
:1096D0002046C9B203B0BDE8F04003F02DBF4C4BAB
:1096E000D6F8030053F8243098474B4B03EB84140F
:1096F00020618AE0464BD6F8030053F8243098479F
:1097000004F0010320219940024641F01101600854
:10971000C9B251E5D6F803102046C9B203B0BDE87E
:10972000F04003F09EBED6F803102046C9B203B045
:10973000BDE8F04004F047B9D6F803102046C9B29E
:1097400003B0BDE8F04004F0EDB8334B03EB8414F4
:10975000D6F80330237258E02D4BD6F8030053F8A7
:1097600024309847A4012C4B18514EE0284BD6F8D2
:10977000030053F824309847274B03EB84146060B0
:1097800043E0254BD6F8032003EB84135A8307E00C
:10979000D6F80310204603B0BDE8F04004F0EEBB5D
:1097A000204603B0BDE8F04004F025BB1A4B03EBA4
:1097B0008414D6F80330236227E0D6F803308BB147
:1097C000012B1DD1144A02EB84121376104B134A5D
:1097D00043F8242003EB8404114B2365114B2363CE
:1097E000114B0BE00C4A02EB84121376084A0F4B24
:1097F00042F8243002EB840423652363A36604E06B
:10980000042200E003220A4B1A7003B0F0BD00BF2F
:109810007886FF1F5096FF1F0094FF1FFDDC00009D
:1098200061DD000039DD0000A1DD0000C9DD0000C0
:109830006898FF1F38B5CF4DCF4CA8786B780528B6
:1098400002D90423237038BDA42B00F0428200F219
:10985000B080112B00F0CF814FD8082B00F06E8123
:1098600029D8032B00F03E810ED8012B4FEA50027D
:1098700000F0010100F0218100F22A81202303FA87
:1098800001F141F00D011DE1052B00F04181C0F017
:109890003981062B00F04481072B40F0CC8200F088
:1098A00001032021994041F010014008C9B203F0A2
:1098B0007FFCC0B240E10C2B00F0668107D80A2B78
:1098C00000F0498100F24E8104F006FAFEE00E2B12
:1098D00000F07981C0F068810F2B00F08181102B9E
:1098E00040F0A982A54B03EB800320211D6D00F001
:1098F0000103994041F00501FEE01A2B00F0C181FF
:109900002FD8152B00F0938113D8132B4FEA500258
:1099100000F00101994D4FEA800000F0778100F2DC
:109920007E812844202303FA01F1856E41F00A016B
:1099300073E1172B00F08D81C0F08081182B00F0AF
:109940009381192B40F0778200F001032021994088
:1099500041F014014008C9B203F02AFCC0F38000B2
:10996000B4E01F2B00F0A0810ED81C2B00F09981D1
:10997000C0F094811D2B40F05E82804B03EB80038E
:109980001D6D02F079FCBBE08C2B00F09A8107D8AA
:109990007F2B40F05082794B184490F8483048E2D1
:1099A000A22B00F09381A32B40F0458203F05CFED4
:1099B0008CE0BB2B00F0E08139D8AD2B00F0B181F9
:1099C00017D8A82B00F0A18105D8A62B00F08F8115
:1099D00040F2828196E1AA2B00F09D81C0F098812F
:1099E000AB2B00F09B81AC2B40F0258203F062FF93
:1099F0006CE0B42B00F09E810BD8B12B00F0948169
:109A0000B32B00F09481AE2B40F0158203F05FFF82
:109A10005CE0B62B00F0A281C0F09781B82B00F07B
:109A2000A881B92B40F0078203F0DDFD4EE0CA2B80
:109A300000F0C58122D8C22B00F0A7810CD8BD2B25
:109A400000F0A081C0F09B81C12B40F0F4814C4B11
:109A500003EB8010037AECE1C42B00F0A881C0F086
:109A60009C81C52B00F0A581C92B40F0E48100F05A
:109A700001032021994041F018019EE1D02B00F014
:109A8000C2810AD8CE2B00F09F8100F2A881CC2B96
:109A900040F0D18103F0C9FF18E0D22B00F0C08163
:109AA000C0F0BB81D42B00F0C081FF2B40F0C381FC
:109AB000334B03EB8010037EBBE1202303FA01F15B
:109AC00041F001011046C9B203F072FB6060B4E1DD
:109AD0002A4B03EB8000202303FA01F1056D41F0CE
:109AE00007019AE0254B03EB800320211D6D00F058
:109AF0000103994041F002014008C9B203F058FB4C
:109B0000A847E3E71D4B03EB8000036D80694CE140
:109B10001A4B1C4A03EB800352F820009B6E44E171
:109B200000F001032021994041F010014008C9B222
:109B300003F03EFBC0F30720C000C7E700F00103BD
:109B40002021994041F015014008C9B203F030FBD3
:109B5000C0F34020BAE700F001032021994041F012
:109B6000150117E000F001032021994041F0150193
:109B700020E000BF5096FF1F6898FF1F7886FF1FE8
:109B80000094FF1F3096FF1F00F001032021994031
:109B900041F014014008C9B203F00AFB10F0020FB3
:109BA00014BF0023012344E100F001032021994068
:109BB00041F014014008C9B203F0FAFA00F00100C4
:109BC00080F0010082E700F001032021994041F07C
:109BD00014014008C9B203F0EBFAC0F3001075E7B6
:109BE0009E4B03EB800320219D6E00F00103994002
:109BF00041F0040180E7994B03EB800320219D6E27
:109C000000F00103994041F0080175E72844202342
:109C100003FA01F1056D41F0030110466DE7284498
:109C2000202303FA01F1056D41F00B01F5E700F087
:109C300001032021994041F00C01BEE0874B03EB6A
:109C4000800320211D6D00F00103994041F01201B5
:109C500052E7824B03EB800320211D6D00F00103CE
:109C6000994041F0130147E700F00103202199409A
:109C700041F014014008C9B203F09AFAC0F3C000E1
:109C800024E700F001032021994041F0140140082D
:109C9000C9B203F08DFAC0F3C02017E703F0CAFC85
:109CA00014E703F0D4FC11E700F0010320219940F0
:109CB00041F010014008C9B203F07AFAC0F3034042
:109CC00004E703F09DFCC0F10800FFE603F07EFC12
:109CD000FCE603F0E3FCF9E603F0C6FC18B9A8784B
:109CE00003F067FCF2E6A87803F0E5FCEEE603F08B
:109CF000BBFC18B9A87803F04FFCE7E6A87803F09E
:109D0000ECFCE3E603F031FCE0E603F0F1FDDDE618
:109D100003F0B6FDDAE603F0C0FDD7E603F0A3FDDD
:109D2000D4E603F0F2FDD1E603F077FCCEE603F0D3
:109D3000E1FCCBE600F001010901400841F06F01B0
:109D400003F036FAC0F30440C0E6444B444A03EB48
:109D5000800302EB80101B6D006926E03F4B03EB94
:109D6000800320211D6D00F00103994041F0110195
:109D7000C2E603F086FCA9E603F07BFEA6E603F04C
:109D800084FEA3E603F08CFEA0E6344B344A03EBDA
:109D9000800380011B6D105807E0304B304A03EB05
:109DA000800302EB80101B6D406898478EE62D4BB8
:109DB00000E02D4B53F820303BE0400883E6284B71
:109DC00003EB8010438B34E000F0010109014008EF
:109DD00041F06F0103F0ECF9C0F3090076E6AB78CF
:109DE000224AD05C0021616010B121480125456004
:109DF000D154204AD15C19B1616841F0020161601F
:109E00000021D15419E000F001010901400841F09E
:109E10006F0103F0CDF9001658E604F0A5F855E6F9
:109E20000F4B03EB8010C36903E00D4B03EB801075
:109E3000036A636001E0032323700F4B1B7863B157
:109E40000E4B62681A600E4B1AB91A6842F008028B
:109E500002E01A6822F008021A6038BD7886FF1FF7
:109E60000094FF1FBC93FF1F8495FF1FF893FF1FF3
:109E70006898FF1FDC93FF1F6398FF1F5498FF1F14
:109E80005896FF1F38B5AC4A9378022B144600F061
:109E9000F980032B00F0FD80002B40F0F98153780E
:109EA0004E2B00F0A2802BD8462B73D016D8422B15
:109EB00061D009D8402B5AD0412B40F0E7819F4B0D
:109EC000D178197000205AE0442B5CD0452B40F02B
:109ED000DD819A4BD1785971052050E04B2B74D01D
:109EE00004D8472B5ED0492B63D0CFE14C2B77D0E1
:109EF0004D2B40F0CB81914BD178597515203EE028
:109F0000542B00F0998019D8512B7FD009D84F2BB2
:109F100075D0502B40F0BA81884BD17899751620B6
:109F20002DE0522B00F08180532B40F0AF8183490C
:109F3000D2F8033041F8103F102031E0842B00F0BC
:109F400096800BD8552B00F08280832B40F09E81A9
:109F50007B4BD2F80320C3F8802038BD852B00F05E
:109F60008B80FF2B40F09281D278764B92E145F2C4
:109F7000FF70D17803E0714BD17859700120BDE8B2
:109F80003840FEF7C4BE6D49D2F8033041F81C3F9B
:109F90001C2005E06949D2F8033041F80C3F0C2041
:109FA000042260E06549D2F8033041F8083F0820F8
:109FB000F6E7D278614B0AB9DA7503E0624901220B
:109FC000DA754A601720D97DD9E75C4CD178E17009
:109FD0000320FEF79CFEE078BDE83840FEF798BB12
:109FE000564BD17899700220C9E7544CD2F803003F
:109FF000E084FEF78BFD26202118022233E0D2F800
:10A0000003104E4BC9B259761920B8E74B4B1A7D55
:10A0100012F0010F1D4604D0E378DB0701D4FEF7F0
:10A02000E2FEE17829751420A9E74449D2F803300B
:10A0300041F8203F2020B3E7D2F80330012B00F293
:10A0400027813E49D37801F81A3F1A200AE0D2F856
:10A050000330012B00F21C81374B3849DB7801F8C3
:10A060001B3F1B200122BDE83840FEF762BE374B84
:10A07000D2F803201A6038BD314BD2F80320C3F860
:10A08000842038BD5178324BD2F8032043F8212088
:10A0900038BD53782E2B00F2F980DFE813F02F0043
:10A0A00039004300F700F700F700F700F700F7006A
:10A0B0005D00620067006C0071007600F700F70039
:10A0C000F700F700F700F700F700F700F700F700D8
:10A0D000F700F7007B0082008900900097009E0047
:10A0E000A500AC00B300BA00C100C800CF00D40086
:10A0F000D900DE00E300E800ED00F200154BD4F8D3
:10A1000003201A60FEF78EFA0D4BC3F8880038BDA5
:10A11000104BD4F803205A60FEF784FA084BC3F8BA
:10A120008C0038BD0B4BD4F803209A60FEF77AFA06
:10A13000034BC3F8900038BD5096FF1F0C80FF1FE3
:10A140007886FF1F6298FF1F6898FF1F6498FF1FA3
:10A150007498FF1F9C95FF1F4F4BD4F80320DA60C3
:10A1600038BD4D4BD4F803201A6138BD4A4BD4F8A2
:10A1700003205A6138BD484BD4F803209A6138BD9A
:10A18000454BD4F80320DA6138BD434BD4F80320A3
:10A190001A6238BDD4F803203F4BD2B283F8242092
:10A1A00038BDD4F803203C4BD2B283F82A2038BD06
:10A1B000D4F80320384BD2B283F8252038BDD4F828
:10A1C0000320354BD2B283F82B2038BDD4F80320BE
:10A1D000314BD2B283F8262038BDD4F803202E4B61
:10A1E000D2B283F82C2038BDD4F803202A4BD2B247
:10A1F00083F8272038BDD4F80320274BD2B283F848
:10A200002D2038BDD4F80320234BD2B283F8282068
:10A2100038BDD4F80320204BD2B283F82E2038BDAD
:10A22000D4F803201C4BD2B283F8292038BDD4F8CF
:10A230000320194BD2B283F82F2038BD164BD4F827
:10A2400003201A6338BD144BD4F803205A6338BD79
:10A25000114BD4F803209A6338BD0F4BD4F8032078
:10A26000DA6338BD0C4BD4F803201A6438BD0A4BAE
:10A27000D4F803205A6438BD074BD4F803209A64FD
:10A2800038BD054BD4F80320DA6438BD032200E062
:10A290000422024B1A7038BD9C95FF1F6898FF1F5F
:10A2A0002DE9FF41C64EC74F32787A7064233B7068
:10A2B000212AD6F803307B6035463C4601F0928077
:10A2C0005AD80E2A00F0CA842AD8072A00F03D8303
:10A2D00011D8032A00F0888107D8012A00F0BE8037
:10A2E000022A00F0118101F06BBB052A00F02583E2
:10A2F00040F2A58125E30A2A00F02F8309D8082A15
:10A3000000F02383092A41F05B83FFF7BBFD01F0D6
:10A3100059BB0C2A00F05D8440F2448400F06FBC0D
:10A32000182A00F0098612D8142A00F02D8507D8C3
:10A330000F2A00F0B284132A00F0ED8401F040BB34
:10A34000162A00F0E18540F24F8500F0E2BD1C2A9C
:10A3500000F0408706D81A2A00F0108640F2FD85EA
:10A3600000F01DBE1F2A00F0898700F2D4871E2A44
:10A3700000F0358701F024BB802A01F01F8138D816
:10A38000402A01F009811BD8242A01F094800DD8BD
:10A39000222A01F08980232A41F012838A4B1B680C
:10A3A000C6F80330FFF76EFD01F00CBB262A01F062
:10A3B000B980C1F0AD80272A01F0DC8001F000BB3C
:10A3C000442A01F0F28008D8422A01F0E88001F224
:10A3D000E98001F048FF01F0F5BA462A01F0EB8070
:10A3E000C1F0E680472A41F0EB8201F042FF01F024
:10A3F000E9BA872A01F0B48117D8832A01F0FA80DC
:10A400000BD8812A01F0DF80822A41F0D9826F4B7C
:10A41000022283F8942001F0D5BA852A01F01D812B
:10A420006B4A41F2098101F02BB98C2A01F0F081CD
:10A4300009D8892A01F0BE81C1F05D818A2A01F024
:10A44000D08101F0BDBAF22A01F06C82FF2A01F03E
:10A45000AE828D2A41F0B48201F0FEB9B378052BAB
:10A4600055D85C4A5C4E0024D4545C4AD454F25C07
:10A4700072B103F0010220219140594A41F00601D6
:10A48000580852F82320C9B202F062FEAB78F454A7
:10A49000AC78544BD5F8030001271F554B4B0028CF
:10A4A000B8BF404253F824309847202604EA0701F9
:10A4B00006FA01F141F007010246C9B224FA07F099
:10A4C00002F046FED5F80330A878002B0DDD00EA37
:10A4D000070306FA03F100228DE88400F840C9B2B0
:10A4E000134602F0F9FD01F06DBA00F0010306FA1F
:10A4F00003F1002202238DE80C004008C9B2134684
:10A5000002F0EAFD01F05EBAB378052B03D904230B
:10A51000237001F057BA2F4A2F4E0024D4542F4AEB
:10A52000D454F25C7AB103F00102202191402C4A0C
:10A5300041F00601580852F82320C9B202F008FE83
:10A540001F4B9B78F454AC78264BD5F803000127B9
:10A550001F551E4B0028B8BF404253F8243098477F
:10A56000202604EA070106FA01F141F0070102463C
:10A57000C9B224FA07F002F0EBFDD5F80330A87851
:10A58000002B0EDD00EA070306FA03F10022022386
:10A590008DE80C00F840C9B2134602F09DFD01F0B1
:10A5A00011BA00F0010306FA03F100228DE88400DD
:10A5B0004008C9B2134602F08FFD01F003BA00BF94
:10A5C0005096FF1F6898FF1F5498FF1F7886FF1F43
:10A5D0000C80FF1FDC93FF1F4896FF1FF893FF1F9F
:10A5E0003096FF1FE293FF1FB07805288FD802F046
:10A5F0007BFBB0789D4B012200EA0201202404FA83
:10A6000001F141F007011A54C9B2D040002202F012
:10A610009FFDB07800F0010104FA01F1022300244B
:10A6200001932246234600944008C9B202F054FD2B
:10A63000B3788F4AD4548F4AD45401F0C3B9B07858
:10A64000052804D98C4A5278022A41F0BB81884AF5
:10A65000894F00261654874A16546A78012A49D031
:10A6600003D3022A00F0AF8063E1804C235C7BB10E
:10A6700000F0010320219940804B03EB800341F05F
:10A6800007019A694008C9B202F062FDBB78E6543E
:10A69000AB787B4CE25C82B103F001022021914057
:10A6A000784A41F0060152F823205808C9B202F056
:10A6B0004FFD714B9B780022E254A878D5F8032017
:10A6C000202400F0010104FA01F141F00D014008DD
:10A6D000C9B202F03DFDA87800F00103002204FA9F
:10A6E00003F1009201924008C9B2134602F0F4FC53
:10A6F00001F068B9614A1318904693F84830012B6D
:10A700000CD004D3022B14D103F02EFC10E000F087
:10A7100001032021994041F00D0105E000F0010303
:10A720002021994041F001014008C9B202F040FDEA
:10A730000646A8784D4F3B5C83B100F00103202111
:10A74000994008EB800341F007019A694008C9B2BB
:10A7500002F0FEFC484B9B780022FA54AB78484F3D
:10A76000FA5C82B103F0010220219140454A41F098
:10A77000060152F823205808C9B202F0E9FC3E4B0A
:10A780009B780022FA54A878D5F8033000F0010134
:10A79000202707FA01F11E4441F00D014008C9B21B
:10A7A000324602F0D5FCA87800F00103002207FA37
:10A7B00003F1009201924008C9B2134602F08CFCEA
:10A7C000666001F0FFB8142B00F3AF8003065FD57D
:10A7D0003446AB782341DF0742D5DFF8908014F888
:10A7E0000830670804F001066BB12021264BB14008
:10A7F00041F0070153F82420F8B2C9B202F0A8FCD6
:10A80000002304F80830DFF8788014F808306BB1C2
:10A8100020211C4BB14041F0060153F82420F8B22E
:10A82000C9B202F095FC002304F80830202303FA93
:10A8300006F6D5F80330062202FB0342134BFFB2A3
:10A8400046F00D0153F822203846C9B202F080FCD0
:10A850000022009201923846F1B2134602F03CFC0D
:10A860000134062CB5D101F0ADB800BFE293FF1F53
:10A87000DC93FF1FF893FF1F5096FF1F7886FF1F82
:10A880004896FF1F3096FF1F9086FF1F5C96FF1FA4
:10A8900005284AD8A44C235C7BB100F00103202199
:10A8A0009940A24B03EB800341F007019A694008ED
:10A8B000C9B202F04DFCBB78E654AB789C4CE25C2C
:10A8C00082B103F00102202191409A4A41F0060131
:10A8D00052F823205808C9B202F03AFC964B9B78F4
:10A8E0000022E254A878D5F80330202400F00101BA
:10A8F000062202FB030204FA01F1904B41F00D0124
:10A9000053F822204008C9B202F022FCA87800F0D7
:10A910000103002204FA03F1009201924008C9B237
:10A92000134602F0D9FB01F04DB80423237001F067
:10A9300049B80323237001F045B8FEF7EFFA01F0A0
:10A9400041B8FEF777FF01F03DB8B378052B3FF62D
:10A95000DEAD0323237001F035B8B378022B00F08D
:10A96000AC80032B00F0AE80002B40F003817378A5
:10A97000502B71D027D8472B62D013D8422B55D0FB
:10A9800007D8402B4CD0412B40F0F2806C4B1B7809
:10A990004EE0452B4ED050D8442B40F0E980684B18
:10A9A000DB6945E04C2B50D007D8492B4AD04B2BC4
:10A9B00040F0DE80624BDB783AE04E2B604B47D0B4
:10A9C00048D85B7D34E0802B55D014D8532B49D028
:10A9D00007D8512B43D0522B40F0CA80584B1B6AEA
:10A9E00026E0552B44D040D3562B40F0C180544B29
:10A9F00093F824301CE0832B48D008D8812B3ED01C
:10AA0000822B40F0B580494BD3F8983010E0852B6D
:10AA100042D03FD3FF2B40F0AB804A4B1B7848E03D
:10AA200045F2FF70FEF7AFF97860A5E0444B5B7824
:10AA30006360A1E0424B5B79FAE7414BDB68F7E7E3
:10AA40003F4B6BE03E4BDB7D33E03D4B9B78EFE7CC
:10AA5000DB8CEDE75B7EEBE7394B9B7DE8E7384B22
:10AA60001B7DE5E7364B1B69E2E7354B9B7EDFE755
:10AA7000334BDB7EDCE72D4B93F89430D8E72B4B40
:10AA800093F894301E1F73427341D1E7274BD3F8DC
:10AA90008030CDE72C4B3EE0244A2C49D2F884305C
:10AAA0004B4303F540533933C2F8843023F000435D
:10AAB000BEE7003318BF0123BAE77278244B53F87E
:10AAC0002230B5E77378282B2AD011D8022B24D056
:10AAD00005D8FBB1012B4BD11E4B5B68A8E7092BB6
:10AAE00046D30E2B48D9272B42D11A4B1B6B9FE71D
:10AAF0002B2B34D006D8292B2ED02A2B38D1154B0E
:10AB0000DB6B95E72D2B30D02CD32E2B30D1114B76
:10AB1000DB6C8DE70F4B1B688AE70E4B9B6887E762
:10AB20000C4B5B6B84E700BFE293FF1F7886FF1F2F
:10AB30004896FF1F3096FF1F5096FF1F5C96FF1F21
:10AB40000C80FF1F6298FF1F6498FF1F6D4EC64167
:10AB50007498FF1F9C95FF1F9C4B9B6B68E79B4B5A
:10AB60001B6C65E7994B5B6C62E7984B9B6C5FE7EE
:10AB7000032300E004232370954B1B78002B00F087
:10AB80002187944B62681A60934B2AB91A6842F085
:10AB900008021A6000F016BF1A6822F008021A6054
:10ABA00000F010BFB378022B0FD18C4B5B78372BA2
:10ABB0003FF6CFAE8A4903F5FF70800001EB8301B9
:10ABC0000422FEF7B6F800F0FDBE04233B7000F04F
:10ABD000F9BEB378022B0ED17378372B3FF6B9AE9E
:10ABE0007F4903F5FF70800001EB83010422FEF72B
:10ABF000DCF800F0E7BE04233B7000F0E3BEB07861
:10AC000005283FF684AC754B5B78012B07D002D347
:10AC1000022B08D01EE002F05FF800F0D3BE02F075
:10AC200063F800F0CFBE02F067F8694B78601B78DC
:10AC3000002B00F0C786674B1860674B1A6820B975
:10AC400042F008021A6000F0BDBE22F008021A604D
:10AC500000F0B8BE03233B7000F0B4BEB278022A05
:10AC600017D17078072808D81BB9FDF795FE00F0BA
:10AC7000A9BEFDF77DFE00F0A5BEFF2840F0A2862C
:10AC80005D1C0ABF534BD8B21878FDF799FE00F04F
:10AC900099BE04233B7000F095BEB378012B1CD005
:10ACA0002BB1022B1FD17078FDF7B4FE13E0707842
:10ACB000082802D8FDF795FE0DE00A2807D1494B78
:10ACC0001B6983F40073C3F340237B600DE0FF280E
:10ACD0000BD1FDF7BDFE606007E07078092804D055
:10ACE00002F0A4F8F7E704233B70394B1B78002BE4
:10ACF00000F06886374B62681A60374B2AB91A68C9
:10AD000042F008021A6000F05DBE1A6822F00802E4
:10AD10001A6000F057BE71782E4A092925D8DFE85D
:10AD200001F005080B0E12181B1E212311680B449D
:10AD30001AE01168CB1A17E011684B4314E0116850
:10AD400091FBF3F310E0116891FBF3F003FB101398
:10AD50000AE011680B4007E011680B4304E011683A
:10AD60004B4001E01368DB43136012681A4B2AB9A9
:10AD70001A6842F008021A6000F024BE1A6822F035
:10AD800008021A6000F01EBE124A12689A42124B64
:10AD9000196804DD21F0030141F0040108E00BBF54
:10ADA00021F0060121F0050141F0010141F002010D
:10ADB00019602AB91A6842F008021A6000F002BE4F
:10ADC0001A6822F008021A6000F0FCBD9C95FF1F73
:10ADD0006398FF1F5498FF1F5896FF1F5096FF1F40
:10ADE0007498FF1F80F00F4072780C2A00F2EA85F9
:10ADF000DFE802F007111B252F39444E58626C76AC
:10AE00008000B84A1268140740F1DC85B64AC2F8DF
:10AE1000983000F0D7BDB34A1268100700F1D28510
:10AE2000B14AC2F8983000F0CDBDAE4A1268D107E1
:10AE300040F1C885AC4AC2F8983000F0C3BDA94AB9
:10AE40001268D20700F1BE85A74AC2F8983000F018
:10AE5000B9BDA44A1268570740F1B485A24AC2F8A6
:10AE6000983000F0AFBD9F4A126812F0050F00F055
:10AE7000A9859D4AC2F8983000F0A4BD994A12688D
:10AE8000960740F19F85984AC2F8983000F09ABD25
:10AE9000944A1268950700F09585934AC2F8983055
:10AEA00000F090BD8F4A1268D40640F18B858E4A1F
:10AEB000C2F8983000F086BD8A4A1268900640F1C8
:10AEC0008185894AC2F8983000F07CBD854A1268B5
:10AED000510640F17785844AC2F8983000F072BD7F
:10AEE000804A1268120640F16D857F4AC2F8983098
:10AEF00000F068BD7B4A1268D70540F163857A4A45
:10AF0000C2F8983000F05EBD774AC2F8983000F081
:10AF100059BD754AD2F89C10072900F25385481C88
:10AF200002EB8101C2F89C00D2F89800C1F8A000A1
:10AF3000C2F8983000F046BD6B4BD3F89C20002A35
:10AF400000F04085013AC3F89C2003EB8202D2F85E
:10AF5000A020C3F8982000F035BD73782E2B04D8BC
:10AF6000624A0121D15400F02DBDFF2B7FF4F1ACDA
:10AF70005D4B012283F8C02000F024BD73782E2B96
:10AF800004D85A4A0021D15400F01CBDFF2B7FF495
:10AF9000E0AC554B002283F8C02000F013BD524CAA
:10AFA00094F8C1209AB95E1C4FF00A0205D1504BAB
:10AFB0001B685A43C4F8C42002E05343C4F8C430A9
:10AFC000FDF730FB0123C4F8C80084F8C1306B786A
:10AFD000042B00F2F784DFE803F0034C8DC61D005C
:10AFE000FDF720FBD4F8C820D4F8C4103E4B801ADB
:10AFF00080EAE072A2EBE0728A4204D9002283F870
:10B00000C12000F0DFBCD3F89820013AC3F89820A3
:10B0100000F0D8BCA87801F06FFE40B9314B84F83D
:10B02000C1001A6822F010021A6000F0CBBCD4F8FC
:10B03000C4302D4DB3B1FDF7F5FAD5F8C830D5F8C9
:10B04000C420C01A80EAE073A3EBE073934209D9ED
:10B05000002385F8C130234B1A6842F010021A60B1
:10B0600000F0B0BCD4F89830013BC4F8983000F040
:10B07000A9BCA878202100F00103994041F01501F6
:10B080004008C9B202F094F810F4007609D0002309
:10B0900084F8C130134B1A6822F010021A6000F0D5
:10B0A00091BCD4F8C430104DABB1FDF7BBFAD5F864
:10B0B000C830D5F8C420C01A80EAE073A3EBE0736F
:10B0C000934208D9074B85F8C1601A6842F0100214
:10B0D0001A6000F077BCD4F89830013BC4F898307F
:10B0E00000F070BC5896FF1F7886FF1F0096FF1F68
:10B0F0005498FF1FA878202100F00103994041F0E7
:10B1000015014008C9B202F053F810F0010609D049
:10B11000002384F8C130B94B1A6822F010021A607B
:10B1200000F050BCD4F8C430B54DABB1FDF77AFA9D
:10B13000D5F8C830D5F8C420C01A80EAE073A3EB74
:10B14000E073934208D9AD4B85F8C1601A6842F0AC
:10B1500010021A6000F036BCD4F89830013BC4F8F5
:10B16000983000F02FBCA878202100F0010399400E
:10B1700041F015014008C9B202F01AF810F00206B9
:10B1800009D0002384F8C1309C4B1A6822F01002C9
:10B190001A6000F017BCD4F8C430994DA3B1FDF784
:10B1A00041FAD5F8C830D5F8C420C01A80EAE07357
:10B1B000A3EBE073934207D9904B85F8C1601A68FE
:10B1C00042F010021A60FDE3D4F89830013BC4F855
:10B1D0009830F7E38A4B002283F89420F2E37678E4
:10B1E000142E3FF6B6AB874A9778052F1AD806215A
:10B1F000854C01FB067144F82130844B9B7E002B6B
:10B2000000F0E083002E00F0DD83013E1820704343
:10B21000042200F5D36002FB070004EB8101FDF777
:10B2200088FDCFE3FF2F7FF472A9774F8EB91825E1
:10B23000002405F5D0607919204421440422043407
:10B24000FDF777FD182CF4D11835B5F5FC7FEFD15B
:10B25000B8E300246B7818205A1E5043062202FBE4
:10B26000034100F5D36000EB840007EB8101042269
:10B270000134FDF75EFD062CECD1A3E37378142BAB
:10B280003FF667ABB278052A19D8062101FB0323E4
:10B290005D4951F823205E4B7A601B78002B00F04B
:10B2A00091835C4B1A60554B22B91A6842F0080230
:10B2B0001A6087E31A6822F008021A6082E3FF2A04
:10B2C0007FF425A9504E8BB91825002405F5D060D0
:10B2D00071192044214404220434FDF766FD182C22
:10B2E000F4D11835B5F5FC7FEFD16BE300246B7812
:10B2F00018205A1E5043062202FB034100F5D3607A
:10B3000000EB840006EB810104220134FDF74DFDC2
:10B31000062CECD156E396F801803A4FB8F1140FA1
:10B320003FF617ABBE78300630D50024AB7823410A
:10B33000D90712D5334B20215E7804F001039940E0
:10B3400041F00101C4F34700C9B201F031FF062307
:10B3500003FB06462C4B43F826002C4B9B7E8BB1FF
:10B360006B787BB15A1E182050432749062202FBF6
:10B37000034300F5D36000EB840001EB830104225A
:10B38000FDF7D7FC0134062CD0D11BE3052E3FF688
:10B39000BEA806F001032021994041F00101700888
:10B3A000C9B201F005FF194B174C9B7E062101FB2A
:10B3B000086644F82600002B00F004837B78002BFD
:10B3C00000F00083BD78581E18267043042201FB4C
:10B3D000035100F5D36002FB050004EB8101FDF78A
:10B3E000A8FCEFE272780B4B0A2A50D8DFE802F093
:10B3F00014191F242A32373C41464A005896FF1F31
:10B400007886FF1F5096FF1F5C96FF1F0C80FF1F62
:10B410006398FF1F5498FF1F92491A6809680A44ED
:10B4200003E090491A680968521A1A602FE08D49A2
:10B430001A6809684A43F8E78A491A68096892FB5A
:10B44000F1F2F2E7874A1968126891FBF2F002FB09
:10B450001012EAE7834A11681A680A40E5E7814A50
:10B4600011681A680A43E0E77E4A11681A684A4080
:10B47000DBE77C4A1168C943116008E079491A6822
:10B480000A6004E0774A18681168196010601A6849
:10B49000754B22B91A6842F008021A6092E21A68E3
:10B4A00022F008021A608DE2704B1B68C6F8033068
:10B4B000FDF734FD86E27378052B00F28382DFE826
:10B4C00003F003090F151B21674B1A6802F00F02E6
:10B4D0001A6077E2644B1A6822F010021A6071E277
:10B4E000614B1A6822F020021A606BE25E4B1A6808
:10B4F00022F040021A6065E25B4B1A6822F080027B
:10B500001A605FE2584B1A6822F480721A6059E29E
:10B5100072782E2A3FF61DAA554901EB8202C2F825
:10B52000CC304FE2524B5149D3F888210A604D4943
:10B53000D3F88C210A60D3F890214B49C3F89820A6
:10B54000D3F894210A60D3F8982183F8C120D3F866
:10B550009C21C3F8C820D3F8A021C3F8C4204549D2
:10B5600093F8A421885C08B101208854002283F854
:10B57000A82127E2B378052B3EF6C9AF3E4A5278A0
:10B58000142A3FF6E6A9062101FB0233374A3B495C
:10B59000126841F8232015E200F064FE12E200F088
:10B5A00063FE0FE200F061FE0CE200F05FFE09E2D4
:10B5B00000F05DFE06E200F05BFE03E22C4B002291
:10B5C00083F89420FEE1727812B1012A05D00EE0D2
:10B5D000274B012283F89420F4E1B3F5C05FBEF459
:10B5E00096AF234981F89420C1F89830EAE103230B
:10B5F0003B70E7E11E4B002183F8C01083F8A811CF
:10B600001B4A02F1CC034FF0FF3043F821001948E8
:10B610000023435401312F29F2D182F89430C2F82B
:10B620009830C2F89C3082F8C130104A13600D4A3D
:10B6300013600D4A1360C5E1127D92070AD4B3F579
:10B64000C05FBEF464AF0A4A042182F89410C2F8C5
:10B65000AC31B7E108233B70B4E1054B002283F81D
:10B660009420AFE17098FF1F5896FF1F5498FF1F5A
:10B670007886FF1F0096FF1F5096FF1F5C96FF1FE6
:10B680009849994C927822700125B3F5C05F0D70EE
:10B6900027D2964A127D12EA050622D1184602A93F
:10B6A000FDF79AFB9DF8083063709DF80930A37090
:10B6B0009DF80A30E3709DF80E3023719DF80D302F
:10B6C00063719DF80C30A3719DF80B30E371267205
:10B6D0002B46E15C227A01330A44082B2272F8D10E
:10B6E00070E101230021E1540133082B7E4AF9D196
:10B6F0001378137266E17378012B1DD00AD3022BE5
:10B700002BD1784B01221A70784B774A9B781370B3
:10B71000002319E0734B01221A70744B724A9B7814
:10B720001370734B186800230133C118082B11F8EC
:10B73000011CD154F8D145E11822FA717B714322E2
:10B740000323BA713B713DE16A4901331944082B67
:10B7500011F8091CD154F7D134E103233B7031E1D6
:10B760007378032B00F22E81DFE803F0020F1C2018
:10B77000614B93F89420FA7193F8C120D3F8AC315F
:10B78000BA711A0A7A713B711CE15B4B93F89420F1
:10B79000FA7193F8C120D3F89830BA711A0A7A7105
:10B7A0003B710FE1554B1B687B600BE1544B1B68F1
:10B7B0007B6007E17278002A40F00481B1780029AB
:10B7C00040F0008140F2D242934240F0FB8045F2CB
:10B7D000FF70FDF79CFAFDF706FB0120FDF704F86A
:10B7E000F0E07278474B02B101221A70464BEA78BA
:10B7F0001A70414B93F8B011444B1970444900231F
:10B800000B7044490B70444B19780A431A70D9E005
:10B81000757815B1012D0FD01BE0042245F2FB70A5
:10B8200002A9FDF7C2FA029BD6F803209A4206BF8E
:10B8300001237B607D60C5E0B3782A2B06D145F2F9
:10B84000FB7036490422FDF774FABBE003233B701A
:10B85000B8E003233B70B5E07278032A3ED8DFE8F6
:10B8600002F008022F3A24480022D0F8B41105460D
:10B8700010E0214AD2F8B411092907D8481CC2F8AF
:10B88000B40102EB8102C2F8B8319BE009233B709E
:10B8900098E001328A4200F09580214850F8224019
:10B8A0009C424FEA8206F4D18319481E824204D298
:10B8B0005C6843F8044B0132F7E7C5F8B40181E056
:10B8C0000D4A0023C2F8B431154A002199500433BF
:10B8D000282BF9D176E00A237B6073E003233B70C9
:10B8E00070E000BF5898FF1F5998FF1F0C80FF1F82
:10B8F0000880FF1F008000007886FF1F5498FF1FFC
:10B900007098FF1FD493FF1FE993FF1FFF95FF1F40
:10B91000E893FF1F4E96FF1FD593FF1F5396FF1FFF
:10B920003088FF1F7378812B7EF4F1ADB278274BFE
:10B93000922A7EF4ECAD9A79A32A7EF4E8AD5A7986
:10B94000B42A7EF4E4AD1A79C52A7EF4E0ADDB7842
:10B95000D62B7EF4DCADFDF714F9FCF763FE04464C
:10B96000FCF760FE001B0028B8BF4042B0F57A7FAC
:10B97000F6DBFCF733FF164B00221A604FF0FF3264
:10B98000C3F87021C3F87022C3F87421C3F874227D
:10B99000C3F87821C3F87822C3F87C21C3F87C224D
:10B9A0000C4B0D4A1A600120FCF71EFF0AE040F222
:10B9B000D242934206D1094B012283F8E02101E0F3
:10B9C0000223237004B0BDE8F08100BF5096FF1F32
:10B9D00010E000E00080FF1F785634127886FF1FC9
:10B9E0002DE9F843414B424E00241C60414BC6F800
:10B9F00098401C60404B86F8C1401C6025463F4B78
:10BA000003EB85131A7E3E4BA3F1200003F11801CE
:10BA10002AB93C4A32511A5102510A5107E03A4AB6
:10BA200032513A4A1A513A4B03513A4B0B5105F0F5
:10BA300001034FF0200808FA03F8C5F347095FFA3D
:10BA400088F848F00701484601F0B2FB324B185124
:10BA5000324B0027EF5448F00601484601F0A8FB9E
:10BA60002F4B18512F4BE8B2EF54013502F0C3F9B8
:10BA7000062D04F10404C2D13B462B4A0021995003
:10BA80000433B3F5806FF8D1284FBB7E8BB11825F6
:10BA90000024274905F5D06029442044214404228C
:10BAA0000434FDF782F9182CF3D11835B5F5FC7F75
:10BAB000EED1FB7E13B17B7D9BB10DE04FF4FF64B3
:10BAC0001C49204621440422FDF76FF9043440F656
:10BAD000D8039C42F4D1EEE7FCF7FEFF08B1012346
:10BAE00000E0002386F89430BDE8F8835498FF1FE7
:10BAF0007886FF1F7098FF1F5896FF1F0094FF1F46
:10BB0000C886FF1FC9DD0000FDDC000061DD00000C
:10BB100039DD0000A1DD00009086FF1FE293FF1FCA
:10BB20003096FF1F4896FF1F7498FF1F0C80FF1F61
:10BB30005C96FF1F7C90FF1FF7B50F4C0F4E86469B
:10BB40000F4694E80300C6F803300D4BB270002294
:10BB50008DE803001A7086F800E07770FEF7A0FB0E
:10BB6000084A217882F8E1119DE80300636884E8BF
:10BB70000300184603B0F0BD6898FF1F5096FF1FE2
:10BB80006398FF1F7886FF1FF7B51F4E02460C46CD
:10BB900096E803008DE803001C4953780B709378F6
:10BBA0004B70D3788B7013798B7153794B71937978
:10BBB0000B71D379CB70164B00271F70FEF770FB0B
:10BBC000144B19786D46334671B921706170327823
:10BBD000A2707278E270F2792271B2796271727930
:10BBE000A2713279E27109E0012907D13A460A4986
:10BBF00011444978A1540132082AF8D195E803008C
:10BC000083E8030003B0F0BD6898FF1F5096FF1F44
:10BC10006398FF1F5898FF1F5998FF1F014B93F817
:10BC2000E10170477886FF1F2DE9F043BE4BBF4C02
:10BC30001B7889B063B1BE4B1B78062B08D00A2B4A
:10BC400006D003F0EF030F2B1CBF002384F8B031A4
:10BC500094F8B031B74E032B1FD133788BB9B64F60
:10BC6000B64DB87897F801802A78804490446A7875
:10BC70009044EA799044AA7990446A7990442A7968
:10BC800018E0012B40F08C800025AD4B585D01354C
:10BC9000FCF702FD092DF8D182E0042B28D1A64F34
:10BCA000A64DB87897F80180002301226B702A70A6
:10BCB0006B6080449044FCF7EFFC7878FCF7ECFC78
:10BCC0002878FCF7E9FC6878FCF7E6FCE879FCF7F3
:10BCD000E3FCA879FCF7E0FC6879FCF7DDFC5FFA8F
:10BCE00088F82879FCF7D8FC4046FCF7D5FC57E0EB
:10BCF000072B33D1337802A833BB8F4B93F802C0A4
:10BD000093F801808D4B8DF808C093F800E05F78C0
:10BD1000DD798DF80AE0C444E64499798DF80B701A
:10BD200077445A798DF80C503D441B798DF80D10ED
:10BD300029448DF80E200A448DF80F3013448DF8F5
:10BD400009808DF8103029E0012B27D100237C4A8F
:10BD50009A5CC2540133092BF9D11FE0082B1FD183
:10BD6000764A00230120537010705360724A8DF898
:10BD70000A00917852788DF809200A4402448DF81F
:10BD800008108DF80B308DF80C308DF80D308DF8D3
:10BD90000E308DF80F308DF8102002A8FCF7EEFE63
:10BDA000684B1A789846002A4FD0674B674D1B782E
:10BDB000032B21D0072B44D15F4B2A7898785978F0
:10BDC0008DF81510802301448DF816300A318A232E
:10BDD0008DF814008DF817308DF81B2000230A44CD
:10BDE00005A88DF818308DF819308DF81A308DF8B7
:10BDF0001C20FCF7C3FE24E04F4F2A78B87897F850
:10BE00000190814409F10A099144FCF745FC7878D6
:10BE1000FCF742FC8020FCF73FFC8A20FCF73CFC4E
:10BE20000020FCF739FC0020FCF736FC0020FCF772
:10BE300033FC5FFA89F92878FCF72EFC4846FCF7BA
:10BE40002BFC00232B7088F80030002384F8B031DD
:10BE5000337094F8E03113B10120FCF7C5FC0DF10B
:10BE60000700FCF731FC0646002877D0FCF744FCBD
:10BE700010B1002384F8E23194F8E2119DF8070034
:10BE80002A4A4B1CDBB22144092B84F8E23181F8A9
:10BE9000E30140F0C580002392F8E31182F8E2311B
:10BEA000254A5278914240F0BB801A461F4D05F258
:10BEB000E311595C01330A44082BD2B2F6D195F84C
:10BEC000EB3193422CD11A4B95F8E4211A7095F876
:10BED000E5215A7095F8E6219A7095F8E7219A7154
:10BEE00095F8E8215A7195F8E9211A7195F8EA2137
:10BEF000DA70FCF797FB164B164A186095F8941009
:10BF000000231370032285F8B0214A1E012A85F808
:10BF1000E231114A02D9052918BF012313707FE0CD
:10BF2000042385F8B0317BE06298FF1F7886FF1FFD
:10BF30005096FF1F5898FF1F0C80FF1F6898FF1F27
:10BF40005998FF1F4E96FF1FFF95FF1FE893FF1F95
:10BF5000F495FF1FFE95FF1F6398FF1F05AD284650
:10BF6000FCF7F9FD00283BD033463246E95C01334B
:10BF70000A44082BD2B2F9D19DF81C1091422CD161
:10BF8000A24B9DF815201A709DF816205A709DF846
:10BF900017209A709DF818209A719DF819205A71EF
:10BFA0009DF81A201A719DF81B20DA70FCF73AFBF5
:10BFB000974B984A186000231370072284F8B02129
:10BFC00094F89420511E01291946934B03D9052A50
:10BFD00001D001221FE0197022E084F8B0311FE087
:10BFE00094F894308D4D013B012B19D8D5F8983039
:10BFF000B3F5C05F11D2FCF76FFD70B1D5F89800B2
:10C000008249431CC5F89830FCF7E6FE092385F801
:10C01000B031814B01221A7002E0002384F8943081
:10C0200094F894307D4D042B04D1784E3278170665
:10C0300040F1BD8094F8B03113F0FB0F05D0082B10
:10C0400003D0062B01D0FEF72BF994F8B031092B61
:10C0500040F08480FCF7E6FA704A714DD2F88820EF
:10C060002B68801A80EAE072A2EBE0729A4209D94A
:10C070006C4B1A78012A04BF02221A70FCF7D2FA1C
:10C08000C4F88800FCF7CEFAD4F88C306A68C01A7D
:10C0900080EAE073A3EBE073934209D9614B5A78CD
:10C0A000012A04BF02225A70FCF7BCFAC4F88C00C3
:10C0B000FCF7B8FAD4F89030AA68C01A80EAE073A6
:10C0C000A3EBE073934209D9564B9A78012A04BF37
:10C0D00002229A70FCF7A6FAC4F8900094F8C030D7
:10C0E000002B3BD04D4B93F8A821002A36D14D4967
:10C0F0008B5C022B2FD1494B03F1CC0050F822006E
:10C10000451C26D0484983F8A4210968C3F8881142
:10C1100046490968C3F88C11D3F89810C3F89011F8
:10C120004349C3F898000968C3F8941193F8C11003
:10C13000C3F898110022D3F8C810C3F89C1183F8F3
:10C14000C120D3F8C410C3F8A011012283F8A8219C
:10C1500004E000238B5401322F2AC8D194F8B01187
:10C160002E4B092906D193F89420022A04BF0522F8
:10C1700083F89420D4F8B421284B002A42D009290E
:10C1800040D193F8941001293CD1D3F898000023B2
:10C19000224901F5DC7454F82340A04203D1052361
:10C1A00081F894302EE001339342F1D12AE095F8E2
:10C1B000B03113F0FB0F25D0082B23D0062B21D054
:10C1C000D5F8AC011B4CD6F803306270B0F5C05FF7
:10C1D000636012D23146FCF7F8FDD5F8AC01314668
:10C1E000FCF71CFE30B1D5F8AC310133C5F8AC31E9
:10C1F000652300E00723237004E007232370002356
:10C2000085F8943009B0BDE8F08300BF5096FF1F59
:10C21000F495FF1FFE95FF1F6398FF1F7886FF1F91
:10C220009C95FF1F0096FF1F5498FF1F7098FF1FDB
:10C230005896FF1F6898FF1F704710B5074CFCF712
:10C24000F1F92368C01AB0F5FA7F05D9044B022230
:10C25000DA60FCF7E7F9206010BD00BF749CFF1F97
:10C2600000F00F4070477047704770477047704745
:10C270007047704700000000014B53F820007047E2
:10C280006488FF1F2DE9F047B74DEB69B3B1B74B99
:10C290001C781E4694B9FCF7C5F9B54B1B68C01A4B
:10C2A000EB690028B8BF4042984207D920460134C4
:10C2B00001F0EAFC062CF9D1012333702B6AC3B1DB
:10C2C000AC4B1C781D46A4B9FCF7ACF9AA4BA64AA6
:10C2D0001B68126AC01A80EAE073A3EBE073934212
:10C2E00007D92046013401F0CFFC062CF9D10123F7
:10C2F0002B70A24CFCF796F994F8303004EB8303D2
:10C300009B69C01A80EAE073A3EBE0730A2B2DDD72
:10C31000FCF788F9064694F83000202100F001036C
:10C32000994041F00101C9B2400800F041FF94F882
:10C33000308004EB88050746686B381A04F08CFDE2
:10C340008146A869301A04F087FD0146484604F08A
:10C350008BFE04F0B1F982A3D3E9002304F000FAC4
:10C3600004F098FC44F82800AE616F6394F8300044
:10C37000824F00F00101202606FA01F141F015017B
:10C380004008C9B200F014FF10F0400905463CD047
:10C3900097F8300000F0010106FA01F14008C9B237
:10C3A00000F006FF0138C0B201280AD997F8300022
:10C3B00000F0010306FA03F14008C9B2012200F0BF
:10C3C000C7FE94F830006E4B012600EA06012027D4
:10C3D0001E5407FA01F16B4B41F006011E54C9B21D
:10C3E000F0404FF6FF7200F0B3FE94F8300000EA20
:10C3F00006018F4047F007010022F040C9B200F06B
:10C40000A7FE94F83030604AD654604B94F8300060
:10C410005A4E03EB80129846126982B300F0010174
:10C42000202707FA01F141F002014008C9B200F0EB
:10C43000BFFE96F8303008EB83120028B8BF4042A8
:10C44000126990421BD9F21892F84C20002A36D17A
:10C450004FEA530A03F001039F4047F01407FFB26D
:10C460003946504600F0A4FE394640F480625046FA
:10C4700000F06EFE96F830301E4401231DE094F863
:10C4800030303E4EE21892F84C20C2B14FEA530AC7
:10C49000202703F001039F4047F01407FFB23946FD
:10C4A000504600F085FE394620F48062504600F088
:10C4B0004FFE96F830301E44002386F84C3094F836
:10C4C0005260DFF8CCA05EB9F0B2FCF78AFA0AF845
:10C4D00006000136082EF7D1284B012283F852209E
:10C4E00027260027F8B2FCF77CFA1AF807308342B7
:10C4F0001BD0274B07F10C02F854264B53F822307F
:10C50000022B05D0032B0AD0012B0ED168B106E017
:10C5100058B9214A915D012907D1935505E01E4B79
:10C520009A5D012A04BF02229A550137082F06F1AD
:10C530000106D7D194F8303015F0010104EB030265
:10C540002CD092F85B1000293DD1012182F85B10BC
:10C55000104A1A4492F8242012F0010F29E000BF7B
:10C56000FCA9F1D24D6290400C80FF1FFE95FF1F89
:10C57000F495FF1FB893FF1FEC95FF1F6488FF1F02
:10C58000E293FF1F4896FF1FF893FF1F0094FF1FC1
:10C59000B788FF1F9C95FF1F0096FF1F92F85B0056
:10C5A00088B182F85B10594A1A4492F8242012F09C
:10C5B000020F08D002211B2211FB0323544AD05C36
:10C5C000012808BFD15494F83030E218AE0792F831
:10C5D00061100AD5E9B9012182F861104B4A1A4469
:10C5E00092F82A2012F0010F09E091B1012182F89E
:10C5F0006110464A1A4492F82A2012F0020F08D01D
:10C600000E33434A12F81310012904BF022102F825
:10C61000131015F0800708D094F830303C4A0333EB
:10C62000D15C012904BF0221D154B9F1000F08D017
:10C6300094F83030364A0F33D15C012904BF02210F
:10C64000D15494F83000334E08EB80131B6A002B52
:10C6500035D06D0533D400F00101202505FA01F134
:10C6600041F01901C9B2400800F0A2FD804696F8D9
:10C67000300000F001018D4045F001014008C9B2D1
:10C6800000F096FD96F83030234A02EB8312C0EB9F
:10C690000800126A80EAE078A8EBE07890450ED9AD
:10C6A000184601F0F1FA96F830301C4A0121D154B5
:10C6B0001533174AD15C012904BF0221D154A7B117
:10C6C000174B94F830101A7842FA01F0C0070CD5D5
:10C6D0000120144D00FA01F12970134D2870134800
:10C6E000007810B922EA01021A7094F83000094D5E
:10C6F00000F05EF894F830300133DBB2052B88BFD0
:10C70000002385F83030BDE8F08700BF9C95FF1FFF
:10C710000096FF1F6488FF1F0094FF1FDC93FF1F1C
:10C72000E993FF1FE893FF1F4E96FF1FD493FF1F4F
:10C730002DE9F341DFF8748018F8003004460E4606
:10C74000450800F001076BB12021164BB94041F0BC
:10C75000060153F824202846C9B200F0F9FC002352
:10C7600008F80430202303FA07F7EDB247F0070179
:10C7700086EAE672A2EBE6722846C9B200F0E8FC4F
:10C78000094A0123002E13554FF00002D8BF02239F
:10C790000193F9B200922846134600F09DFC02B0C6
:10C7A000BDE8F0813096FF1FE293FF1F4896FF1F00
:10C7B0002DE9F04F00F0010320269E404508F6B217
:10C7C000044646F0150185B0284600F0F1FCAB4F59
:10C7D0000246A00107EB000C51089CF80830DCF879
:10C7E000049013F0400F02F0010E09D0385801F008
:10C7F000010BC0F1000A5FFA8EF1C9F1000905E0F2
:10C8000057F800A05FFA8EFB01F001011F0603F04C
:10C810003F0820460391029208D501F05DFAD0F15D
:10C82000010338BF00230399029A06E001F054FA8D
:10C83000029A0399031C18BF012308F1FF3007284F
:10C8400000F24082DFE810F008000800080008004D
:10C850000201020102010201894F3B5D013B0E2BE7
:10C8600000F23082DFE813F00F00230027003300CE
:10C87000370040004F005E009300BA00BF002E0258
:10C88000EE0024021E0246F01401284600F090FC3F
:10C8900007EB84077B4A7A4BB8600121A8F10208B4
:10C8A0008845115594BF022204221A550AE207EB6B
:10C8B00084039A6808E1002900F00482284646F0C3
:10C8C000010100F075FC704B43F824001DE107EBFB
:10C8D00084039A6828E1BBF1000F00F0F381204641
:10C8E00001F0D2F90623ECE107EB840328469A68AD
:10C8F00046F0140122F0030200F02AFC20464946CB
:10C90000FFF716FF3BE1BBF1000F40F0DB81204653
:10C910005946FFF70DFF2046C9F10001FFF708FF58
:10C920000823CEE1BBF1000F00F0CC8146F00101FD
:10C93000284600F03DFC002180462046FFF7F8FE27
:10C94000514B53F82420C8EB020243F8242007EB94
:10C95000840328469A6846F0140122F0030200F08E
:10C96000F7FB284646F007014A4600F0F1FB28464F
:10C9700046F00D01424600F0EBFB00221346009208
:10C9800001922846314600F0A7FB092399E1910561
:10C9900040F1988146F0010A5146284600F008FC13
:10C9A0003A4B002118602046FFF7C2FE284646F0A9
:10C9B0000D01002200F0CCFB28465146002200F079
:10C9C000C7FBA8F10308284646F01901002200F031
:10C9D000BFFBB8F1010F00F26981FDE0BBF1000F70
:10C9E00000F0708109E1BBF1000F40F06B8146F06F
:10C9F0000101284600F0DCFB594680462046FFF73F
:10CA000097FE07EB840328469A6846F0140122F04B
:10CA1000030200F09DFB284646F007014A4600F05D
:10CA200097FB0222284646F00D0198FBF2F200F037
:10CA30008FFBCDF800B0CDF804B0284631465A46F9
:10CA40005B4607E1920540F13D812FE10C4F385DD7
:10CA500001380E2800F23681DFE810F01A002E00AF
:10CA60004F005E0080003401930034013401C500A2
:10CA7000D100AA0000012A01240100BF0094FF1F79
:10CA8000CC88FF1FE293FF1FBC93FF1F8495FF1FFD
:10CA90008E4B0122284646F014011A5500F088FBFF
:10CAA00007EB8403B8F1060F986061D0B8F1080F66
:10CAB0005ED00422864BF8E6B8F1060F0AD107EBE8
:10CAC00084039A6822F00302284646F0140142F0DB
:10CAD00002020AE0B8F1080F09D107EB84032846E7
:10CAE0009A6846F0140122F0030200F031FB204660
:10CAF0005146FFF71DFE0323E3E0A8F10502012ADA
:10CB000005D821B1B8F1060F34D10423D9E0002BA8
:10CB100000F0D8800C23D4E0B8F1050F0AD107EB60
:10CB200084039A6822F00302284646F0140142F07A
:10CB300001020AE0B8F1070F09D107EB8403284688
:10CB40009A6846F0140122F0030200F001FB20462F
:10CB5000CAF10001FFF7ECFD0523B2E0A8F10502E0
:10CB6000012A09D8BBF1000F06D0B8F1050F01D199
:10CB70000223A6E00F23A4E0002B00F0A3800723EC
:10CB80009FE0002B40F09E80A8F10708B8F1010F4C
:10CB90000BD907EB840328469A6822F0030246F07B
:10CBA000140142F0020200F0D3FA2046494616E092
:10CBB000002B40F08780A8F10708B8F1010F0BD9CE
:10CBC00007EB840328469A6822F0030246F014011A
:10CBD00042F0010200F0BCFA2046C9F10001FFF763
:10CBE000A7FD0A236DE0002B6CD0284646F001011A
:10CBF00000F0DEFA07EB840318620B2361E0002BE0
:10CC000060D146F0010107EB84082846039300F049
:10CC1000CFFAD8F80820824646F01401284622F0C0
:10CC2000030200F095FA284646F007014A4600F054
:10CC30008FFAD8F8202092440222284646F00D01AF
:10CC40009AFBF2F200F084FA039B009301932846CA
:10CC500031461A4600F040FA0D2332E0930531D5F3
:10CC60000E233B5546F001073946284600F0A0FA4E
:10CC7000184B002118602046FFF75AFD284646F061
:10CC80000D01002200F064FA28463946002200F027
:10CC90005FFA284646F01901002205B0BDE8F04FC2
:10CCA00000F056BA20460021FFF742FD0E2308E0AF
:10CCB00007EB840328469A6846F0140100F048FA0E
:10CCC00000233B5505B0BDE8F08F00BFE293FF1F86
:10CCD000CC88FF1F8495FF1F024B1A5C0AB9012202
:10CCE0001A547047CC88FF1F024B1A5C0AB10F22FE
:10CCF0001A547047CC88FF1F014B185C704700BF67
:10CD0000CC88FF1F104A684620F0070113698D4642
:10CD100040F273214B434FF6FF71B3FBF1F36E2BDF
:10CD200001B504D9094B4FF48021596005E04F2B20
:10CD300003D8064B4FF480219960BDE8014057238A
:10CD400013608546704700BF00B0034080F00F407D
:10CD50001F4B68461A6820F007018D4602F01F023B
:10CD600001B5072A2DD8DFE802F0040A2C10161CA2
:10CD700022281969174A89B21180412222E01969D3
:10CD8000144A89B2518043221CE01969114A89B2C0
:10CD9000D180442216E019690E4A89B211814522D8
:10CDA00010E019690B4A89B2518146220AE01969DB
:10CDB000084A89B29181472204E01969054A89B27B
:10CDC000D1814022BDE801401A608546704700BF0E
:10CDD00000B00B400489FF1F38B541F23002114BFF
:10CDE000995841F00061995041F23C020024995851
:10CDF00041F00061995003F5E8230D2540229D6024
:10CE00004920DC605C621A6001F01AFB064B572275
:10CE10009D602720DC605C621A60BDE8384001F04C
:10CE20000FBB00BF0070044000B003400B2829D89E
:10CE3000DFE800F006090D10282828281328191EFD
:10CE4000114B188901E0104B588980B270470E4B86
:10CE50009889FAE70C4BD889F7E70B4B588840F2D2
:10CE6000732380B208E0084BD8888E2380B203E099
:10CE7000054B1888422380B258434FF6FF7390FB4E
:10CE8000F3F07047002070470489FF1F684620F0C8
:10CE900007018D4611B53D4BDA7842F00202DA7097
:10CEA0003B4A1078C0B20228114641D0032835D041
:10CEB000012867D1547891788C4216D2D978C90765
:10CEC00009D451785068C9B24C1CE4B25470425C29
:10CED000D2B21A7156E0997801F0DF019970997811
:10CEE00001F0EF01997010724AE0517A01F0FF00F1
:10CEF00049B9997801F0DF019970997801F0EF0153
:10CF0000997010703EE0997841F004019970917A1F
:10CF1000C9B2197100235372032332E0997801F0EA
:10CF2000EF0199701B79D168DBB20B70022328E006
:10CF3000147C507C84421FD2507C127C821A012ABD
:10CF400005D19A7802F0DF029A7000230B704A7CB8
:10CF50000B7CD31A022B04DC0C4B9A7842F00802AB
:10CF60009A700B7CCA68DBB2581CC0B208740749BF
:10CF70000979C9B2D15405E0997801F0DF019970BF
:10CF800000231370BDE811408546704700700640CD
:10CF90001489FF1F0B4A41F234031920D15841F084
:10CFA0008001D150084B4FF400729A62DA6203F5A7
:10CFB000E0331B225A70C0229A7000225A7101F08D
:10CFC0003FBA00BF0070044000B0044010B5124BDF
:10CFD0000024D2B21C725C729A7001225C701A70CA
:10CFE0000E4A5960917801F0F7019170917841F003
:10CFF00010019170917800F0FE0041F020019170D5
:10D0000010711A78002AFCD1034B187AD0F1010074
:10D0100038BF002010BD00BF1489FF1F00700640FC
:10D0200010B5124B0024D2B21C725C725A740322E7
:10D030001C741A700E4AD960917801F0F701917052
:10D04000917841F010019170917840F0010041F029
:10D050002001917010711A78002AFCD1034B187AC4
:10D06000D0F1010038BF002010BD00BF1489FF1FA0
:10D070000070064070B5164C0025E36001269DF84F
:10D0800010302572D2B26672A2706570637440EA85
:10D0900006032574A3720F4B616026709A7802F024
:10D0A000F7029A709A7842F010029A709A7800F01B
:10D0B000FE0042F020029A7018712378002BFCD1F8
:10D0C000034B187AD0F1010038BF002070BD00BFBB
:10D0D0001489FF1F007006402DE9F0471F461A4BC8
:10D0E0009DF8206033F810409DF82450904681460A
:10D0F0008A46002241F080012046FBF797FD414619
:10D1000000222046FBF792FD394600222046FBF71D
:10D110008DFD0AF07F0A314600222046FBF786FD8E
:10D1200047EA08272946204601220AEB4A0AFBF76C
:10D130007DFD46EA0726D144044B45EA062543F81F
:10D140002950BDE8F08700BF781701002889FF1F2C
:10D15000F8B5154B33F81050144606460F4600221A
:10D1600041F080012846FBF761FD210E0022284690
:10D17000FBF75CFDC4F3074100222846FBF756FD90
:10D1800007F07F07C4F3072100222846FBF74EFD76
:10D1900007EB47072846E1B20122FBF747FD3E4473
:10D1A000024B43F82640F8BD781701002889FF1F7D
:10D1B000294B70B501F07F055A19127B002A43D024
:10D1C00033F81040294600222046FBF72FFD0021AE
:10D1D0000A462046FBF72AFD00210A462046FBF7B7
:10D1E00025FD00210A462046FBF720FD00210122F3
:10D1F0002046FBF71BFD00210A462046FBF716FDE3
:10D2000000210A462046FBF711FD002106020A46CE
:10D210002046FBF70BFD0021304306020A4620465C
:10D22000FBF704FD30430602002120460122FBF7F4
:10D23000FDFC222D46EA000001D0422D0AD1030256
:10D2400008D540F07F4070BD05EB45052844034BF1
:10D2500053F8200070BD00BF781701002889FF1F18
:10D26000F8B50E4C04440D4694F800269AB900F027
:10D270000106360146F06C064708F6B231463846DC
:10D28000FFF796FF05F00F0320F00F0231463846F6
:10D290001A43FFF75DFF84F80656F8BD2889FF1F83
:10D2A00070B500F00104240144F06C044508E4B2B8
:10D2B0000E4628462146FFF77BFF06F0070220F0C6
:10D2C00070032146284643EA0212BDE87040FFF78A
:10D2D0003FBF70B500F00104240144F06C04450820
:10D2E000E4B20E4628462146FFF762FF06F00F0221
:10D2F00020F4F0632146284643EAC212BDE870409C
:10D30000FFF726BF70B500F00104240144F06C045F
:10D310004508E4B20E4628462146FFF749FF06F0CD
:10D32000030220F4C0332146284643EAC232BDE856
:10D330007040FFF70DBF70B500F00104240144F008
:10D340006C044508E4B20E4628462146FFF730FF3C
:10D3500006F00F0220F470032146284643EA0252E9
:10D36000BDE87040FFF7F4BE70B500F00104240181
:10D3700044F06C044508E4B20E4628462146FFF707
:10D3800017FF06F00F0220F070632146284643EA9B
:10D390000262BDE87040FFF7DBBE70B500F001042B
:10D3A000240144F06C044508E4B20E4628462146A8
:10D3B000FFF7FEFE16B140F0804201E020F080420F
:10D3C00028462146BDE87040FFF7C2BE70B500F0A8
:10D3D0000104240144F06C044508E4B20E462846DA
:10D3E0002146FFF7E5FE16B140F4002201E020F4EB
:10D3F000002228462146BDE87040FFF7A9BE70B55F
:10D4000000F00104240144F06C044508E4B20E4627
:10D4100028462146FFF7CCFE16B140F4802201E0F9
:10D4200020F4802228462146BDE87040FFF790BED8
:10D4300070B500F00104240144F06C044508E4B226
:10D440000E4628462146FFF7B3FE16B140F480424F
:10D4500001E020F4804228462146BDE87040FFF7F5
:10D4600077BE70B500F00104240144F06C04450857
:10D47000E4B20E4628462146FFF79AFE16B140F464
:10D48000005201E020F4005228462146BDE87040D9
:10D49000FFF75EBE70B500F00104240144F06C0497
:10D4A0004508E4B20E4628462146FFF781FE16B134
:10D4B00040F4805201E020F4805228462146BDE825
:10D4C0007040FFF745BE70B500F00104240144F040
:10D4D0006C044508E4B20E4628462146FFF768FE74
:10D4E00033074CBF20F0700320F4076306F00702F7
:10D4F00048BF43F400632846214643EA0212BDE8D0
:10D500007040FFF725BE70B500F00104240144F01F
:10D510006C044508E4B20E4628462146FFF748FE53
:10D5200006F00F0220F4F0632146284643EAC212B7
:10D53000BDE87040FFF70CBE70B500F00104240197
:10D5400044F06C044508E4B20E4628462146FFF735
:10D550002FFE16B140F4003201E020F400322846DC
:10D560002146BDE87040FFF7F3BD08B5094B034401
:10D5700093F8002652B900F00101090141F06C0155
:10D580004008FFF715FE00F00F0008BD93F80606EF
:10D5900008BD00BF2889FF1F00F00101090108B57F
:10D5A00041F06C01C9B24008FFF702FEC0F302105F
:10D5B00008BD00F00101090108B541F06C01C9B2D4
:10D5C0004008FFF7F5FDC0F3C31008BD00F00101EE
:10D5D000090108B541F06C01C9B24008FFF7E8FD48
:10D5E000C0F3C13008BD00F00101090108B541F0E8
:10D5F0006C01C9B24008FFF7DBFDC0F3035008BD62
:10D6000000F00101090108B541F06C01C9B2400800
:10D61000FFF7CEFDC0F3036008BD00F00101090172
:10D6200008B541F06C01C9B24008FFF7C1FDC0F375
:10D63000807008BD00F00101090108B541F06C01DE
:10D64000C9B24008FFF7B4FDC0F3C04008BD00F008
:10D650000101090108B541F06C01C9B24008FFF7AA
:10D66000A7FDC0F3804008BD00F00101090108B525
:10D6700041F06C01C9B24008FFF79AFDC0F3803059
:10D6800008BD00F00101090108B541F06C01C9B203
:10D690004008FFF78DFDC0F3403008BD00F00101E8
:10D6A000090108B541F06C01C9B24008FFF780FDDF
:10D6B000C0F3003008BD00F00101090141F06C0128
:10D6C00008B5C9B24008FFF773FDC0F302130205A5
:10D6D00048BF43F00803184608BD00F001010901E6
:10D6E00008B541F06C01C9B24008FFF761FDC0F315
:10D6F000C31008BD00F00101090108B541F06C013B
:10D70000C9B24008FFF754FDC0F3404008BD70B5F2
:10D7100000F00104240144F06D044508E4B20E4613
:10D7200028462146FFF744FD06F0030220F060037F
:10D730002146284643EA4212BDE87040FFF708BD83
:10D7400070B500F00104240144F06D044508E4B212
:10D750000E4628462146FFF72BFD06F0030220F473
:10D76000C0432146284643EA4232BDE87040FFF7F5
:10D77000EFBC70B500F00104240144F06D044508CD
:10D78000E4B20E4628462146FFF712FD06F00F02CE
:10D7900020F470632146284643EA0222BDE8704027
:10D7A000FFF7D6BC70B500F00104240144F06D040D
:10D7B0004508E4B20E4628462146FFF7F9FC06F07C
:10D7C0000F0320F00F02214628461A43BDE870409F
:10D7D000FFF7BEBC70B500F00104240144F06D04F5
:10D7E0004508E4B20E4628462146FFF7E1FC20F446
:10D7F0007F022146284642EA0642BDE87040FFF714
:10D80000A7BC70B500F00104240144F06D04450884
:10D81000E4B20E4628462146FFF7CAFC16B140F492
:10D82000004201E020F4004228462146BDE8704055
:10D83000FFF78EBC70B500F00104240144F06D04C4
:10D840004508E4B20E4628462146FFF7B1FC16B162
:10D8500040F0807201E020F0807228462146BDE849
:10D860007040FFF775BC00F00101090108B541F0F7
:10D870006D01C9B24008FFF79BFCC0F3411008BD21
:10D8800000F00101090108B541F06D01C9B240087D
:10D89000FFF78EFCC0F3413008BD00F00101090123
:10D8A00008B541F06D01C9B24008FFF781FCC0F333
:10D8B000032008BD00F00101090108B541F06D0128
:10D8C000C9B24008FFF774FC00F00F0008BD00F07B
:10D8D0000101090141F06D0108B5C9B24008FFF727
:10D8E00067FC0314D8B21B0648BF60F0FF0008BDF8
:10D8F00000F00101090108B541F06D01C9B240080D
:10D90000FFF756FCC0F3C03008BD00F0010109016B
:10D9100008B541F06D01C9B24008FFF749FCC0F3FA
:10D92000006008BDF8B510F001064FEA50040F463C
:10D9300020460CBF10211821FFF73AFC07F0030224
:10D9400020F44015002E204645EA02520CBF10215B
:10D950001821BDE8F840FFF7FBBB70B510F00106D9
:10D960004FEA50040D4620460CBF10211821FFF746
:10D970001FFC15B140F4802201E020F48022002E2B
:10D9800020460CBF10211821BDE87040FFF7E0BB16
:10D99000F8B510F001064FEA50040F4620460CBFC0
:10D9A00010211821FFF704FC07F0030220F4403592
:10D9B000002E204645EA02420CBF10211821BDE886
:10D9C000F840FFF7C5BB70B510F001064FEA5004F0
:10D9D0000D4620460CBF10211821FFF7E9FB002E51
:10D9E00020F47F4242EA052220460CBF1021182174
:10D9F000BDE87040FFF7ACBB70B510F001064FEA10
:10DA000050040D4620460CBF10211821FFF7D0FB13
:10DA1000002E20F0FF0242EA050220460CBF102132
:10DA20001821BDE87040FFF793BB10F0010F08B557
:10DA30000CBF102118214008FFF7BAFBC0F30150BA
:10DA400008BD10F0010F08B50CBF102118214008C7
:10DA5000FFF7AEFBC0F3804008BD10F0010F08B522
:10DA60000CBF102118214008FFF7A2FBC0F30140B2
:10DA700008BD10F0010F08B50CBF10211821400897
:10DA8000FFF796FBC0F3072008BD10F0010F08B5A3
:10DA90000CBF102118214008FFF78AFBC0B208BD57
:10DAA00010F0010F08B514BF192111214008FFF72C
:10DAB0007FFBC0B208BD2DE9F743FAF7B3FD04467A
:10DAC000FAF7B0FD001B0028B8BF40420928F7DD77
:10DAD0000027FCB201264FF03509002520466C21B5
:10DAE000002233464FF014088DE84002FFF7F4FAA5
:10DAF000204630212A460723CDF800800195FFF704
:10DB0000EBFA20467C212A4633468DE84002FFF797
:10DB1000E3FA0723204650212A46CDF800800195DC
:10DB2000FFF7DAFA204629462A46FFF711FB20467E
:10DB300020212A46FFF70CFB20462D212A46FFF71D
:10DB400007FB204621212A46FFF702FB2046402101
:10DB50002A46FFF7FDFA20464D212A46FFF7F8FA3C
:10DB6000204641212A46FFF7F3FA20462321324678
:10DB7000FFF7EEFA20462421DC22FFF7E9FA2046DF
:10DB8000252146F6DB02FFF7E3FA2046262140F284
:10DB9000B712FFF7DDFA204627214DF2B712FFF743
:10DBA000D7FA2046282140F2B712FFF7D1FA2046D3
:10DBB0002A21DC22FFF7CCFA20462B210A22FFF78C
:10DBC000C7FA204643213246FFF7C2FA20464421D5
:10DBD000DC22FFF7BDFA2046452146F6DB02FFF7BF
:10DBE000B7FA2046462140F2B712FFF7B1FA2046B5
:10DBF00047214DF2B712FFF7ABFA2046482140F219
:10DC0000B712FFF7A5FA20464A21DC22FFF7A0FA57
:10DC1000374420464B210A22FFF79AFA032F7FF45C
:10DC200058AFE8B2FFF7A1FC054B5855063B002260
:10DC3000EA540135062DF4D103B0BDE8F08300BFEE
:10DC40002E8FFF1F38B5074C044494F8001641B9D5
:10DC500094F80656FFF704FB012384F8003684F895
:10DC6000065638BD2889FF1F064B034493F800264B
:10DC700032B1002293F8061683F80026FFF7F0BAB7
:10DC8000704700BF2889FF1F73B5114B012600EABA
:10DC9000060120241E548C400E4BC0F34705E4B20D
:10DCA0001E5444F0070128460022FFF751FA284687
:10DCB00044F006014FF6FF72FFF74AFA00228DE8A2
:10DCC0004400284621461346FFF706FA02B070BD0D
:10DCD000E293FF1F4896FF1F10F0010F08B54FF0A9
:10DCE00004014FEA500004D0FFF762FAC0F340107D
:10DCF00008BDFFF75DFAC0F3001008BD002808B5A5
:10DD000009DB02F0C7FC0AA3D3E9002302F052FEAC
:10DD100003F06AFC08E002F0BDFC05A3D3E9002390
:10DD200002F048FE03F0D0FB02F0B4FF08BD00BFD4
:10DD300034F7FFFF7F84EE3F08B502F0ABFC06A38B
:10DD4000D3E9002302F036FE03F04EFC02F0A2FFFE
:10DD500008BD00BFAFF30080EB1100A2941A5D4034
:10DD6000002808B509DB02F095FC0BA3D3E90023DA
:10DD700002F0F6FC03F0A8FB08E002F08BFC06A31F
:10DD8000D3E9002302F0ECFC03F02EFC02F082FF4A
:10DD900008BD00BFAFF3008034F7FFFF7F84EE3F84
:10DDA00008B502F077FC06A3D3E9002302F0D8FC03
:10DDB00003F08AFB02F06EFF08BD00BFAFF30080E6
:10DDC000EB1100A2941A5D40704700BFAFF30080D2
:10DDD00010B50024E0B200F001032021994041F089
:10DDE0001A014008C9B24FF480320134FFF7B0F98C
:10DDF000062CEFD110BD2DE9F347594C04EB8014EC
:10DE0000183463684FEA500900F001080BB16588C7
:10DE1000C5B9202303FA08F85FFA88F85FFA89F990
:10DE200048F0180421464846FFF7C2F9214620F47D
:10DE300080624846FFF78CF9484648F01A014FF4D3
:10DE4000803282E0FFF7DCFBC0F1080005FA00F049
:10DE500002F020FCD4F804A004468AEAEA70A0EBA1
:10DE6000EA700D4602F016FC02460B462046294693
:10DE700002F0A0FD3B4B002204460D4602F070FC70
:10DE80006A4606460F4603F051FA0022002302F0CC
:10DE9000CFFEC0B13946304602F0FCFE202303FA23
:10DEA00008F85FFA88F8BAF1000F5FFA89F948F0CC
:10DEB000180504462946B8BF44424846FFF778F99A
:10DEC00020F4806239E0204629466A4603F02EFAA3
:10DED000BAF1000F04460D46DDE900010CDD02F049
:10DEE000D9FE1DA3D3E9002306042946204602F0EB
:10DEF00037FC02F0CFFE0FE002F0CCFEC04316A3C9
:10DF0000D3E9002306042946204602F029FC02F04A
:10DF1000C1FEC0F51C501030202303FA08F85FFA48
:10DF200088F85FFA89F948F0180540EA060429469E
:10DF30004846FFF73DF940F4806248462946FFF71E
:10DF400007F9484648F01A01224602B0BDE8F047FA
:10DF5000FFF7FEB8AFF30080000000000088C34068
:10DF60000094FF1F0000F04000F0010320219940C1
:10DF700041F019014008C9B2FFF71AB900F00103D6
:10DF80000A462021994041F019014008C9B2FFF723
:10DF9000DFB800BFAFF3008038B504460D4600225D
:10DFA000C4F3471140F20110FAF740FEE10041F0DE
:10DFB000060101F0FE010022240A40F20110FAF7E6
:10DFC00035FE24F01F0141F01001002240F2011043
:10DFD000FAF72CFEE9B2002240F20110FAF726FE11
:10DFE000290A40F201100122BDE83840FAF71EBEAE
:10DFF00010B50446C4F34711002240F20110FAF7AD
:10E0000015FEE10041F0060101F0FE010022240AA4
:10E0100040F20110FAF70AFE24F01F0141F00C0152
:10E02000002240F20110FAF701FEFF21002240F227
:10E030000110FAF7FBFD00210A4640F20110FAF741
:10E04000F5FDFF210446012240F20110FAF7EEFD32
:10E0500044EA002080B210BD38B505460C460022C7
:10E06000C5F3471140F20110FAF7E0FDE90041F075
:10E07000060101F0FE0100222D0A40F20110FAF71C
:10E08000D5FD25F01F0141F01001002240F20110E2
:10E09000FAF7CCFDE1B2002240F20110FAF7C6FD1A
:10E0A000C4F30721002240F20110FAF7BFFDC4F3C8
:10E0B0000741002240F20110FAF7B8FD210E40F2AC
:10E0C00001100122BDE83840FAF7B0BD70B5044632
:10E0D000C4F34711002240F20110FAF7A7FDE10056
:10E0E00041F0060101F0FE010022240A40F2011075
:10E0F000FAF79CFD24F01F0141F00C01002240F2D0
:10E100000110FAF793FDFF21002240F20110FAF707
:10E110008DFD00210A4640F20110FAF787FD00212B
:10E1200005460A4640F20110FAF780FD0021044638
:10E130000A4640F20110FAF779FDFF210646012256
:10E1400040F20110FAF772FD360446EA00602843F7
:10E1500040EA042070BD70B504460D46164662B311
:10E16000C4F34711002240F20110FAF75FFDE1000D
:10E1700041F0060101F0FE010022240A40F20110E4
:10E18000FAF754FD24F01F0140F2011041F0100194
:10E190000022FAF74BFD0024731E9C4240F201104E
:10E1A00005D2295D0022FAF741FD0134F4E7E95C6C
:10E1B0000122BDE87040FAF739BD70BDF8B50446DC
:10E1C0000D46164692B3C4F34711002240F20110E7
:10E1D000FAF72CFDE10041F0060101F0FE010022FA
:10E1E000240A40F20110FAF721FD24F01F0141F04A
:10E1F0000C01002240F20110FAF718FD40F2011064
:10E20000FF210022FAF712FD0024771EBC4240F2E3
:10E21000011006D200210A46FAF708FD28550134FC
:10E22000F3E7FF210122FAF701FDE855F8BD38B503
:10E2300004460D460022C4F3471140F20110E400E9
:10E24000FAF7F4FC44F0040101F0FC01002240F272
:10E250000110FAF7EBFC294640F201100122BDE85B
:10E260003840FAF7E3BC10B50446C4F34711002266
:10E27000E40040F20110FAF7D9FC44F0030101F088
:10E28000FB01002240F20110FAF7D0FCFF2100222E
:10E2900040F20110FAF7CAFC40F20110FF210122FE
:10E2A000BDE81040FAF7C2BC08B5094B19685960BF
:10E2B0001B7A0BB141F010014FF4987089B2FFF74F
:10E2C0006BFE4FF49A700021BDE80840FFF764BE72
:10E2D000348FFF1F08B5094B5968196041F01001D0
:10E2E00001224FF4987089B21A72FFF755FE4FF46D
:10E2F0009A701121BDE80840FFF74EBE348FFF1F12
:10E3000008B5124B4FF400225A601A699205FCD5E9
:10E310004FF4A070FFF76CFEC0B20528F8D10C4B8B
:10E3200001224FF4987011215A601A72FFF734FEDF
:10E330004FF49A700021FFF72FFE4FF401704FF653
:10E340000E71BDE80840FFF727BE00BF40F00F4048
:10E35000348FFF1F38B54FF40870FFF749FEC2072E
:10E3600053D54FF49070FFF743FE284C00F00F0395
:10E370002360C3060DD5237A5BB100254FF4987056
:10E38000A1882572FFF708FE4FF49A702946FFF71F
:10E3900003FE6368013B072B37D8DFE803F0041264
:10E3A0000C1A363636242368022B26D0032B24D0B1
:10E3B000012B26D138BD2368012B1ED0032B20D181
:10E3C00023E02368022B20D0042B16D0012B18D178
:10E3D00013E02368013B072B13D8DFE803F00E0E90
:10E3E00012161212120E2368013B072B09D8DFE820
:10E3F00003F0040408040808080CBDE83840FFF7DF
:10E4000053BFBDE83840FFF765BF38BD348FFF1FED
:10E41000FEE74FF0E023084AC3F8082D074A4CF204
:10E420002053D3814DF62813D381138823F00103A1
:10E430001B041B0C13807047008000000020054067
:10E44000802810B54FF00101154A06DD00F01F00CD
:10E450008140C2F88C11D16010BD402806DD00F06B
:10E460001F008140C2F88811916010BD20280C4621
:10E4700006DD00F01F008140C2F88411516010BD1C
:10E48000084B0340002B03DA013B63F01F03013309
:10E49000034A04FA03F3C2F88031136010BD00BFD1
:10E4A00000E100E01F000080802810B54FF001025D
:10E4B000134905DD00F01F008240C1F88C2010BD1B
:10E4C000402805DD00F01F008240C1F8882010BD03
:10E4D0002028144605DD00F01F008240C1F884208A
:10E4E00010BD084B0340002B03DA013B63F01F0310
:10E4F0000133034A04FA03F3C2F8803010BD00BFB1
:10E5000000E100E01F00008003291ADC202818DC4D
:10E5100004220C4B90FBF2F2D2B2034002F16042B3
:10E520008901002B02F56442C9B203DA013B63F0B2
:10E5300003030133DBB21068DB0001FA03F3184375
:10E540001060704703000080064B1A78D2B2012A8F
:10E5500005D1222902D0212901D100225A7001229D
:10E560005A707047408FFF1F70B5144611B91B4B8E
:10E57000197070BD022903D1184B01221A7070BDA9
:10E58000042914D1154B5B78012B25D195880023E4
:10E59000402D28BF40255E1CDBB2AB4205D222686D
:10E5A000D05C00F0C7F83346F5E7002007E0032908
:10E5B0000CD10A4B5A78012A0ED100209870022102
:10E5C00002460346BDE8704000F046BF052903D16E
:10E5D000024B00221A705A7070BD00BF408FFF1F9F
:10E5E00010B50446204600F0BDF80028FAD110BD51
:10E5F000704710B5084C02460B4600200121A1705F
:10E6000000F0EEFA224618B10023A370122010BDCC
:10E610009378002BFCD110BD408FFF1FF8B5064644
:10E620000F4600F0FAFC0E4B1A78012A16D15B78DF
:10E63000012B13D100F000F988B10025ECB2BC42E7
:10E6400005D330462146BDE8F840FFF7D2BF301968
:10E6500000F0D6F801350028F0D0F2E70C20F8BD24
:10E66000408FFF1F08B540210248FFF7D7FF00F099
:10E6700095F808BD438FFF1F38B5054600F0A8F890
:10E680000B28044609D106484021FFF7C7FF28B9E7
:10E690002846BDE8384000F09BB80024204638BD2D
:10E6A000838FFF1FF8B5002406460F462546A3B208
:10E6B0009F4207D0305DFFF7DFFF002818BF0B2512
:10E6C0000134F4E72846F8BD38B5451E002415F896
:10E6D000010F28B1FFF7D0FF002818BF0B24F6E781
:10E6E000204638BD07B50123002000930549064B9D
:10E6F000024600F01FFA002814BF1B20002003B0C0
:10E700005DF804FB69E5000049E5000038B50D46F9
:10E71000044600F097F885420AD825440020AC4210
:10E7200007D020B914F8010B00F052F8F7E738BD14
:10E730000B2038BD10B50A4B197840290ED05A78F5
:10E740009C180132D2B2402AA07001F101014FF0B1
:10E750000000197014BF5A70587010BD0B2010BD06
:10E76000C38FFF1F10B50C4B197891B193F842205D
:10E770009C180132D2B2A4780470402A4FF00000F5
:10E7800001F1FF31197014BF83F8422083F8420071
:10E7900010BD0A2010BD00BFC38FFF1F014B1878AA
:10E7A000704700BFC38FFF1F024B1878C0F14000B5
:10E7B000C0B27047C38FFF1F034B00225A7083F80B
:10E7C00042201A70704700BFC38FFF1FFFF7F4BFCE
:10E7D00010B50A4B197840290ED05A789C1801328E
:10E7E000D2B2402AA07001F101014FF0000019706F
:10E7F00014BF5A70587010BD0B2010BD0690FF1F3B
:10E8000010B50C4B197891B193F842209C18013245
:10E81000D2B2A4780470402A4FF0000001F1FF3119
:10E82000197014BF83F8422083F8420010BD0A20FB
:10E8300010BD00BF0690FF1F014B1878704700BF46
:10E840000690FF1F024B1878C0F14000C0B270471D
:10E850000690FF1F034B00225A7083F842201A7063
:10E86000704700BF0690FF1FFFF7F4BF70B5044666
:10E87000007801F08DF901780023DAB28A4208D2DB
:10E8800003EB8305054466786D78AE4203F101031E
:10E89000F3D1154D207A342303FB0253D97810B9F4
:10E8A00098780130987034235A43AB189B788B4288
:10E8B0000DD003F003030C2101FB03220A4B1A4481
:10E8C000131D107951791B89926800F091FBD5F8DE
:10E8D0009C3043B1227A002A224614BF052103212D
:10E8E00012F8080B984770BD4C90FF1F2DE9FF47A9
:10E8F0000D4691468DF80F0001F04AF9022D0646AB
:10E9000049D190F800A00024E3B2534504F101047A
:10E9100009DA03EB830333440DF10F005978DA78F9
:10E9200001F0F6F9F0E74FF000085FFA88F7574575
:10E9300027DA07EB870737447C1C6078A37879785F
:10E94000B4F803200090002001900DF10F0001F0B9
:10E95000BDF96378032B05D19DF80F007978184A2B
:10E9600001F03CFA7978A37841F0100141EAC31133
:10E970000DF10F00C9B2002201F0FAF908F1010807
:10E98000D3E7104BD3F89C30B3B19DF80F00294664
:10E990004A46984710E0002DF3D12B463278591C97
:10E9A000DBB29A42EDD9074A342000FB0323002250
:10E9B0009A70DA700B46F1E704B0BDE8F08700BF4B
:10E9C0006DE800004C90FF1F2DE9F0410C7804F039
:10E9D0006004202C1D4638D14C78042C1CD00AD859
:10E9E000012C2ED02DD3022C1FD0032C29D1BDE811
:10E9F000F04100F05FB9212C1BD005D8202C20D18C
:10EA0000BDE8F04100F03EB9222C16D0232C18D1DD
:10EA1000BDE8F04100F046B902241C8014680025CE
:10EA200025701468671C17606570BDE8F04100F040
:10EA30005BB9BDE8F04100F01DB9BDE8F04100F060
:10EA40007BB900202880BDE8F081402C06D1054C20
:10EA5000D4F8A04014B1A047BDE8F081CD20BDE8B6
:10EA6000F08100BF4C90FF1F73B50446007801F0A1
:10EA70008FF863680093A27A637A43EA0223ADF8C1
:10EA8000043001780023DAB28A4208D203EB83050E
:10EA9000054466786D78AE4203F10103F3D1164D5B
:10EAA000207A342303FB0253D97810B998780130C7
:10EAB000987034235A43AB189B788B420DD003F0E7
:10EAC00003030C2101FB03220B4B1A44131D107985
:10EAD00051791B89926800F08BFAD5F89C304BB1C4
:10EAE000227A20781AB1052104F1080201E00321FD
:10EAF0006A46984702B070BD4C90FF1F07B5436847
:10EB00000093437A817A43EA0123ADF80430084B3D
:10EB1000D3F89C30024643B1017A007811B1052147
:10EB2000083201E004216A46984703B05DF804FB0F
:10EB30004C90FF1F2DE9F843054688461746994635
:10EB400001F026F802789DF82030013206460021B7
:10EB50002846D2B201F09CF8044630BB284614493E
:10EB6000144A00F08EF93378601CE4B2A34211D944
:10EB700004EB8402324434235C430F4992F801E0F1
:10EB800001F804E00B1992785A7000229A70DA703A
:10EB90000446E8E72846494600F066F8044620B9EE
:10EBA000054BC3F89C80C3F8A0702046BDE8F883ED
:10EBB000EDE80000C9E900004C90FF1F08B5074BC5
:10EBC0000022C3F89C20C3F8A02000F0ADF918B9CA
:10EBD000BDE8084001F072B808BD00BF4C90FF1FAF
:10EBE0002DE9F047914607460D46984600F0D0FFC4
:10EBF00002780024E3B2934207D2013404EB84018B
:10EC0000014411F8041CA942F4D1164A3420584397
:10EC10001118CE788B78F41AE4B2042C02D1C120FA
:10EC2000BDE8F08706F003044FF00C0C0CFB040465
:10EC300014440136F6B227716571C4F80890A4F83F
:10EC40000C80CE70F61AF6B2012E07D1384629464E
:10EC50004A464346BDE8F04700F0CAB90020BDE887
:10EC6000F08700BF4C90FF1F014B002019607047D8
:10EC7000F090FF1F024B0979197100F08DBF00BFA2
:10EC8000F090FF1F13B5002402AA1C80044B42F829
:10EC9000041D0979197100F08DFF02B010BD00BF8D
:10ECA000F090FF1F00201880014B4A88DA807047DF
:10ECB000F090FF1F30B50C4602211980217964883D
:10ECC000084D012C297103D1BDE8304000F08ABF06
:10ECD000022C03D1BDE8304000F090BF0020188026
:10ECE00030BD00BFF090FF1F30B50C4602211980E7
:10ECF00021796488084D012C297103D1BDE8304089
:10ED000000F088BF022C03D1BDE8304000F094BF72
:10ED10000020188030BD00BFF090FF1F044B054A53
:10ED200019791B7A1171137203210A23FFF758BF57
:10ED3000F090FF1F4C80FF1F70B500261E808B785F
:10ED40000E4CC3F340014A00637261F3000203F00A
:10ED50000103A37205462272FFF7E0FF23685BB14F
:10ED6000617A01F0020101F0FF02284611B122216F
:10ED7000324600E021219847002070BDF090FF1F2F
:10ED800008B50246034B12F8080B1B68052198478B
:10ED900008BD00BFFC90FF1F38B5084D04462A1D72
:10EDA000012100F0CDFF20460121802200F0E0FF8C
:10EDB0002B6820780A210022984738BDFC90FF1F5D
:10EDC00037B501210DF10702044600F0B9FF9DF8A7
:10EDD0000730074D802B04D1204601212A7900F00D
:10EDE000C7FF2B6820780B210022984703B030BD65
:10EDF000FC90FF1F436805215A7800F0B9BF73B536
:10EE00000122002405460126002100F081FF33463F
:10EE100021468DE850002846102200F057FF214679
:10EE20002246284600F074FF234621468DE8500014
:10EE30002846102200F04AFF31462846022200F000
:10EE400097FF32462846062100F092FF22462846C8
:10EE5000902100F08DFF044B28781B682146224644
:10EE6000984702B070BD00BFFC90FF1F42783AB9CE
:10EE7000C178C90141F0100101F0900100F078BFA4
:10EE8000704773B50C468DF8070001F0FBF91F4E73
:10EE900034600446002836D110211D4A9DF8070031
:10EEA00000F09CFF122104461A4A9DF8070000F06A
:10EEB00095FF2043C4B21421174A9DF8070000F0C3
:10EEC0008DFF2043C4B21321144A9DF8070000F0BF
:10EED00085FF2043C4B21721114A9DF8070000F0B6
:10EEE0007DFF02AD2043C4B2162115F8010D0D4A75
:10EEF00000F074FF2043C4B201212846032200F031
:10EF000037FF03233371204602B070BDFC90FF1F12
:10EF1000FFED0000F5ED000099ED0000C1ED0000EF
:10EF20006DEE000081ED000037B502AC174B04F820
:10EF3000010D0022102120461A6000F051FF12211D
:10EF40000546204600F04CFF2843C5B21421204658
:10EF500000F046FF2843C5B21321204600F040FFD1
:10EF60002843C5B21721204600F03AFF2843C5B216
:10EF70001621204600F034FF284310F0FF0003D193
:10EF80009DF8070001F08AF903B030BDFC90FF1F27
:10EF900030B585B004AC012104F8090D0DF10E0265
:10EFA000204600F0CDFE204606210DF10F0200F0B4
:10EFB000C7FE9DF80E30802B16D19DF80F309B07B1
:10EFC00012D59DF8070000F0E1FD012805460BD1A0
:10EFD00072B6204600F038FB0022204629468DF804
:10EFE0000E2000F0C5FE62B69DF80E0005B030BDE3
:10EFF00073B50E4615461C468DF80700FFF7C8FF8F
:10F00000802807D00DF1070031462A46234600F03C
:10F01000B9FA00E0002002B070BD7047062812D88F
:10F0200080000129C0B204BF0230C0B2074AC0F359
:10F030004703122101FB03231A884FF6FF739A42FC
:10F0400008BFFF207047FF20704700BF0491FF1FDB
:10F050002DE9F041334D344C344E002785F80071D2
:10F060004FF4107284F8400288462046FF2102F0D7
:10F0700013F9304639464FF48062C4F8446202F016
:10F080000BF995F80C3143F0800385F80C3195F8B5
:10F090000C21244B1206FAD4254AFF21117093F853
:10F0A0000C2142F0400283F80C21A3F52C331A689E
:10F0B000B8F1000F02D042F0004201E022F000421D
:10F0C0001A60184B320A02F0FE0283F89C20C6F345
:10F0D000074283F8B020360E164A83F8B460C4F8AD
:10F0E0004822102283F80821012283F89420BF22AD
:10F0F00083F8802093F8002102F07F0283F800213A
:10F1000093F8842042F0010283F8842093F884204D
:10F1100042F0100283F8842084221A770020BDE890
:10F12000F08100BF002007400491FF1F009EFF1FD9
:10F130005680FF1F00A0FF1F0D4B93F80C2102F01B
:10F14000BF0283F80C21BF2283F8802093F884202B
:10F1500002F0FE0283F8842093F8942002F0FE026D
:10F1600083F894201A7F02F07B021A770020704700
:10F17000002007402DE9F3410B460D788C78454976
:10F1800003C902AE06E90300B3F80310B1F5007F2E
:10F1900003D90021D97002211971062D19D8AF00A9
:10F1A000012CF9B201D10231C9B249083A484FF0F5
:10F1B000120C0CFB01FC00EB0C014FF6FF76B1F8D2
:10F1C0000080B045064604D193F80180B8F1030FE2
:10F1D00001D995205BE0012CFBD891F80F80B8F1A4
:10F1E000FF0F04BF4FF0000881F80F80B3F80380D1
:10F1F00020F80C808A73CA7BD6F84802C1F8020056
:10F2000002F0010247EA44071743FFB2CF735A786E
:10F210004A74D6F844220C7402EBC70CB3F803808E
:10F22000ACF80280CCF804004FF0080C02F837C0AC
:10F23000CF7BB3F8038087F0010702EBC70CCCF853
:10F240000400ACF802804FF0480C02F837C0B3F865
:10F2500003703844C6F8480234B9C97B12F831004B
:10F2600060F07F0002F8310058780C4A02AB03EBE3
:10F2700084042DB254F8083C12F82510012818BF58
:10F2800043F001030B43DBB202F82530002002B04B
:10F29000BDE8F081041801000491FF1FC020074061
:10F2A000084610B51146FFF7B9FEFF281CD00F4BDA
:10F2B0001222C0F3470002FB0030D3F84432C27B75
:10F2C00013F8324004F07F0403F8324082F0010169
:10F2D00013F8312002F07F0203F831204FF0FF33A2
:10F2E0008372C372002010BDC42010BD0491FF1FA3
:10F2F00073B50D468DF80700084611461646FFF710
:10F300008DFEFF2804461FD0294632460DF1070026
:10F31000FFF7C6FFC4F3470312210D4C594363188E
:10F32000D4F848221888121AC4F848222DB2094A83
:10F33000002002F825004FF0FF3262545A709A7094
:10F34000DA701A715A7100E0962002B070BD00BFE9
:10F350000491FF1FC02007402DE9F04180460E4672
:10F36000084611461746FFF759FE0C4CC0F34700FC
:10F37000122303FB0040C57BFF2D0DD03A464046CB
:10F380003146FFF78DFF2DB2D4F8443213F8352003
:10F3900062F07B0203F83520BDE8F0810491FF1F85
:10F3A00010B5084600211446FFF738FE084B12221C
:10F3B000C0F3470002FB0030D3F84432C27B03EBBA
:10F3C000C2035A68136823605368636010BD00BFAE
:10F3D0000491FF1F10B508460C461146FFF71EFEAC
:10F3E000FF281AD024B2104B13F82430DBB213F0EC
:10F3F0000C0F12D09B0712D40C4BD3F8443213F8E5
:10F400003020D2090DD180F00100C0B213F83030A5
:10F41000DB090CBF0020032010BD052010BD01201A
:10F4200010BD032010BD00BFC02007400491FF1F86
:10F4300008B5FFF7F3FD074B1222C0F3470002FBAC
:10F440000030C27BFF2A04D0D3F84432002103F8F5
:10F45000321008BD0491FF1F2DE9F041084600213C
:10F460001E461746FFF7DAFD244BC0F3470012256E
:10F4700005FB0035EC7BFF2C3CD0B5F80080D3F8C1
:10F4800044121FFA88F24FF6FF739A4232D084F08A
:10F49000010311F83330C3F3C013D8B250BB4FEAA5
:10F4A000C40C8EB901EB0C033046A3F80280D5F8EA
:10F4B00002205A6011F8343003F0400363F0770300
:10F4C00001F83430BDE8F0812B736B7301EB0C0352
:10F4D0006E81964228BF1646C5F806705E805F6052
:10F4E00011F8343003F0400363F0770301F834304F
:10F4F000BDE8F0819420BDE8F08100BF0491FF1FBA
:10F500002DE9F04107460C46084611461546FFF71F
:10F5100085FD1A4BC0F34700122606FB003618463D
:10F52000F17BFF2927D022B2154B84B196F811C088
:10F53000012D14BF18261426BCF1010F18BF46F088
:10F54000010613F822C046EA0C0603F8226013F8FD
:10F5500022606FF3410603F82260D0F844320022A3
:10F5600003F831203DB9384621462A462B46BDE8EE
:10F57000F041FFF771BFBDE8F08100BF0491FF1FAC
:10F58000C02007402DE9F84308460F460121904668
:10F590009946FFF743FDFF2832D01B4AC0F34700CE
:10F5A000122404FB0024D2F84452E67B15F83630CE
:10F5B000DB0905EBC60223D139B2144B13F8211035
:10F5C00001F0020101F0FF00D1B92188C4F80680E2
:10F5D0001FFA89F363818B42A8BF0B4620736073C7
:10F5E0005380C2F804800FB9C82305E015F83630FF
:10F5F00003F0400363F0770305F83630BDE8F88385
:10F600009320BDE8F88300BF0491FF1FC02007408E
:10F61000034B044883F8981001210A4600F0A8BB68
:10F62000002007404493FF1F054B0648002283F843
:10F630009420802283F80C210121FF2200F098BB46
:10F64000002007404493FF1F38B51A4B93F8002160
:10F6500002F07F0283F8002193F80C2102F0DF0210
:10F6600083F80C2193F8802042F0200283F8802058
:10F6700093F8842002F0DF0283F8842093F894202A
:10F6800002F0DF0283F8942093F8942042F0040201
:10F6900083F8942044F620641D46013CA4B200F097
:10F6A0009DFE002CF9D195F8943003F0FB0385F80A
:10F6B000943038BD002007402DE9FF47BA4CBB4DC0
:10F6C00094F84022039995F8803095F8847095F865
:10F6D00090608DF80420002262F31721039101212C
:10F6E0008DF8062002928DF807208DF80C201F401F
:10F6F0000DEB0102FF2304F510708DF801308DF839
:10F70000053000F01DFB95F80C31D907F6B20FD586
:10F710009DF80130802B0BD195F8003103F07F0369
:10F7200085F8003195F80C3103F0DF0385F80C31D2
:10F730007A0711D59D4B042093F8A41093F8A020CC
:10F7400083F8800004AB42EA012223F80E2D122038
:10F7500001A9029300F056FBFB0749D5934D92484F
:10F760000123BF2785F8803085F8887095F894309C
:10F77000002643F0020385F89430FF2185F8986055
:10F780004FF4107285F8006101F086FD31464FF4A8
:10F790008062D4F8440201F07FFDD4F8443203F5CE
:10F7A0000073C4F84832824BFF221A7095F89430E7
:10F7B00003F0FD0385F8943095F80C3143F04003D5
:10F7C00085F80C319F2385F88C7085F8843095F886
:10F7D000943003F0DF0385F89430102001A900F085
:10F7E00011FB95F8943003F0DF0385F8943061E164
:10F7F0003D0740F1F4806D4B082283F880203209E8
:10F80000C6F3C001062A8DF805208DF8071007D829
:10F81000C6F3800303EB820319B10233DBB200E0CD
:10F82000FF23D4F84452D90068185A084FF0120C3C
:10F830000CFB0244426802924088ADF80D00E07B68
:10F8400080F00100E07383F0010615F83330C3F354
:10F85000801383F001039B0105F836309DF80730D3
:10F860009DF80590012B05EBC60843D1DFF840A1B8
:10F87000B9F1000F14D19AF80090B9F1000F0FD12F
:10F88000FF2349464A4601A88AF80030FFF708FDE1
:10F8900005F8369001A849464A464B46FFF7DCFD7D
:10F8A0009AF80030012B04D09DF80530002B00F0B1
:10F8B0008A80BDF80DC0A38960892288D4F806101B
:10F8C00063449BB29842A38106D85FFA8CFC6245E0
:10F8D0000CD1A47B012C09D11944C31A9342D8BF7F
:10F8E0009AB2A8F80220C8F8041053E00291ADF8CB
:10F8F0000D3068E0B9F1000F1DD16B5CC3F38303D9
:10F900000D2B2B4B06D101218DF806101278D20950
:10F910001A7010E01A78012A0DD1FF21197001A880
:10F920004946FFF7BDFC05F8369001A849464A460E
:10F930004B46FFF791FD62894FF6FF739A4242D022
:10F94000BDF80D00A1892388014489B29842A181A4
:10F9500001D18A4209D86AB3B2FBF3F003FB10204D
:10F9600080B238BBA07B012824D1521A9A42D8BF5A
:10F9700093B243B9D4F80220C8F8042088F80230C2
:10F9800088F8033006E0D4F80620A8F802301144C5
:10F99000C8F8041015F8363003F0400363F077031D
:10F9A00005F8363014E000BF0491FF1F0020074027
:10F9B0005680FF1FD4F8063002934FF0FF33ADF8A6
:10F9C0000D10A372E3729DF8050001A900F01AFA68
:10F9D0003A4B93F8942002F0DF0283F89420B807A2
:10F9E00017D5364C022384F8803094F8883094F888
:10F9F0008C201620134001A98DF80C3000F002FA7B
:10FA0000BF2384F8883094F8943003F0DF0384F83F
:10FA10009430F9061CD5294C202384F8803010231B
:10FA200084F88030142001A900F0ECF994F80C312E
:10FA300043F0200384F80C3194F8003143F0800344
:10FA400084F8003194F8843043F0200384F8843043
:10FA5000BA060DD5194C202384F88030132001A953
:10FA600000F0D0F994F8843003F0DF0384F8843098
:10FA70003B061FD5FF2301A810210DF102028DF8CE
:10FA8000053000F05DF99DF80230012B04D1002211
:10FA90008DF805208DF80730084C802384F88030DD
:10FAA000172001A900F0AEF994F8943003F0DF03B9
:10FAB00084F8943004B0BDE8F08700BF0020074010
:10FAC0000B4611461A4601F0E7BB00BF30B50329CB
:10FAD000039D049C1CD123B9164A2A60042222806B
:10FAE00026E040F209418B4205D1022A4FF0000383
:10FAF00003D9012201E001231A460F490C2000FB23
:10FB00000313D9681B6951F8221029609B5C0EE031
:10FB1000072901D9CD2030BD074B03EB8102126AC2
:10FB20002A60002AF6D003EB4101B1F8403023806F
:10FB3000002030BD5780FF1F0C180100012904D898
:10FB4000034B5B5C137000207047CD20704700BFF3
:10FB50005093FF1F01299DBF024B00205A54CD2016
:10FB6000704700BF5093FF1F01298CBF0020012068
:10FB70007047054B1A788A4204D05878431A584285
:10FB800058417047012070475093FF1F0020704775
:10FB9000004870475C180100012906D8044BC1EBEE
:10FBA000C1011944116000207047CD20704700BF8B
:10FBB0005B80FF1F012910B50DD8094BC1EBC101B6
:10FBC000194408231068C45CC81801330F2B00F8CF
:10FBD000084CF7D101E0CD2010BD002010BD00BFC2
:10FBE0005B80FF1F012905D8034B03EB4101116026
:10FBF00000207047CD2070475293FF1F012905D880
:10FC0000034B03EB4101116000207047CD2070478A
:10FC10005693FF1F01290AD80648136800EB4101DB
:10FC20001B788B7013685B78CB7000207047CD20F9
:10FC3000704700BF5093FF1F01290AD80648136878
:10FC400000EB41011B788B7113685B78CB7100204E
:10FC50007047CD20704700BF5093FF1F084B5A7864
:10FC60001A700023074AFF2199540133072BF9D159
:10FC70000023054A052199540133072BF9D1704718
:10FC80005A93FF1F5C93FF1F6393FF1F00BF7047D2
:10FC9000013AD2B2062A38B505461C4609D8064BA9
:10FCA0005A70FFF7DBFF28462146BDE83840FFF7D2
:10FCB000CFB9992038BD00BF5A93FF1F024B0022D5
:10FCC0005A70FFF739BA00BF5A93FF1F37B50F4C70
:10FCD000257805B9B9B98DF802308DF800109DF876
:10FCE0001830ADF8032000789DF81C208DF8013005
:10FCF0006946FFF73FFA9DF800302BB120B9237811
:10FD0000013B237000E0952003B030BD5A93FF1FE4
:10FD100038B50A4B0C461D7859788D421D4600D1E6
:10FD20004CB900782146FFF7E3FA2CB120B92B78C3
:10FD300001332B7038BD962038BD00BF5A93FF1F8A
:10FD40004B1E062B03D8094B19444B7808E0CB0611
:10FD500009D501F00F01062905D8044B19444B7A47
:10FD60001370002070478220704700BF5A93FF1F16
:10FD70004B1E062B2DE9F0418046154603D8164B45
:10FD800019444A7021E0CB0622D501F00F04062C5D
:10FD90001ED8012A4FEAD1160F4F04D12146324610
:10FDA000FFF7DAFA0FE072B93B195B7A012B0AD13F
:10FDB00021463246FFF7A4FB2CB94046214686F087
:10FDC0000102FFF79DFB3C4465720020BDE8F08115
:10FDD0008220BDE8F08100BF5A93FF1F00207047CA
:10FDE000062903D9A1F11003072B07D8044B53F8B8
:10FDF0002130002B14BF0020C4207047C42070475E
:10FE000084180100102838B504460D4601D1FFF7CB
:10FE100025FF044B53F824300BB1284698470020A7
:10FE200038BD00BF841801001FB504A9144601F8AD
:10FE3000090D02221A8008460DF10F020521FFF775
:10FE40007FFF034B9DF80F201A80236004B010BD84
:10FE50006C93FF1F1FB504A9144601F8090D012278
:10FE60001A8008460DF10F020421FFF769FF044BC9
:10FE70009DF80F201A800020236004B010BD00BF41
:10FE80006C93FF1F7FB500241C8049888DF8070004
:10FE9000ADF80E10FFF768FE00B3BDF80E20114E4E
:10FEA000131B5A425A410DF107000121FFF760FF71
:10FEB0009DF80E200DF107000421FFF759FF73682C
:10FEC0000DF10E02054601219DF807009847736861
:10FED0009DF8070002212246984700E004252846A5
:10FEE00004B070BD6C93FF1F37B502AA002402F85E
:10FEF000010D0D461C80104601210422FFF738FF3A
:10FF00006A88024B20461A7203B030BD6C93FF1F03
:10FF100037B54C888D888DE80C00210AE2B22B465B
:10FF2000FFF7D4FD03B030BD2DE9F04186B00F4698
:10FF30001E4600238DF80F000593904603230DF114
:10FF40000F00012104AA8DF81030FFF7F9FE3D786B
:10FF5000274C15F0030525D106210DF111020DF1F5
:10FF60000F00FFF7EDFE9DF811309DF80F0003F034
:10FF70000303238005AB00930DF1120301930221CB
:10FF80002B462A46FFF7A2FD059BDB7913F0400FB5
:10FF9000238814BF43F0010323F0010323800223CD
:10FFA00033801FE0012D09D19DF81020BB88012A64
:10FFB00002D113F0FF0F14D10023EFE7022D11D16E
:10FFC000397941F010010DF10F00C9B20DF11202A3
:10FFD000FFF7B6FE9DF8123003F001032380358051
:10FFE00000E0CD20C8F8004006B0BDE8F08100BFB9
:10FFF0006C93FF1F7FB500221A800B784E788DF826
:020000021000EC
:10000000070013F003030D46C6F3400632D1B6B124
:100010004B88013B9BB2012B50D80DF10700062104
:100020000DF10F02FFF78CFE0446002847D1AA7895
:100030009DF80F3006FA02F21A43D2B211E04E8850
:10004000012E3BD10DF1070006210DF10F02FFF744
:1000500077FE044698BBAA789DF80F30964023EAB5
:1000600006020DF1070006218DF80F20FFF780FE34
:10007000044624E0022B21D109798DF80F100DF1EF
:10008000070041F010013246FFF772FE6B78002E38
:100090000CBF08210721012B044607D19DF80F1042
:1000A00001F00F00C909FFF7C3F90821054B9DF8BE
:1000B00007005B680DF10F02984700E0CD24204651
:1000C00004B070BD6C93FF1F10B500241C800B782A
:1000D00003F00303012B0A4605D109799278FFF753
:1000E00039FD204610BD042010BD38B50C7804F051
:1000F0000304012C154607D11C80044C09792246C3
:10010000FFF71CFD2C6038BD042038BD6C93FF1F29
:1001100013B5CD298DF8070006D10DF10700902108
:100120000122FFF725FE18E00D481C88018A12689D
:100130008C4288BF198004461B889DF80700002167
:10014000FEF756FF94F90A30002B06DA00210DF174
:1001500007000A460B46FFF77FF902B010BD00BF4B
:100160006C93FF1F73B5054600266A4601218DF882
:1001700000600196FFF7E4FDAA783F4C012A46D1C2
:1001800068680368C4F80A304368A07AC4F80E307F
:1001900004F10A0110F0600F238A13D1E37A374883
:1001A00050F82340002C5ED09DF80020022A5AD837
:1001B00003EB43031844024492F83430012B52D12C
:1001C000287818E0202BADF802301AD873B1020657
:1001D0000CD40A68C4F812204A68C4F816202846CD
:1001E000314604F11A02FFF737F943E0E46B002CC3
:1001F00039D02878224901AA0DF10203A04701460F
:1002000032E002A82B7800F8073D902113E09DF81A
:100210000030042B12D12B78217A02AD05F8063D6F
:100220002846FFF7F5F901210A462846FFF7A0FD09
:10023000227A28460321FFF79BFD1BE094F90A3040
:10024000002B17DBEB78ABB9E66B66B1B5F809307C
:1002500028780833ADF8023004F1120101AA0DF13B
:100260000203B047CBE7CD21287801AA0DF10203A4
:10027000FFF74EFF02B070BD6C93FF1FE418010042
:100280007693FF1F034B5960DA630021024AFFF7A0
:10029000A5BD00BF6C93FF1F6501010007B502AB50
:1002A000054A03F8010D002118465160D163FFF79C
:1002B00097FD03B05DF804FB6C93FF1F00207047AF
:1002C000354B41F24802995821F00F0141F00201EB
:1002D000995041F20402995841F48021995041F219
:1002E0003402995841F48021995003F52C33602150
:1002F00093F8942042F0020283F89420C02283F8FD
:100300000021FF221A7483F8802083F8882083F864
:100310008420002283F88C2083F80C111F491A7561
:10032000080A00F0FE0083F8982083F8C02083F8C4
:10033000C42083F8C82083F8CC2083F8D02083F829
:10034000D42083F8D82083F8DC2083F8E02083F8D9
:10035000E42083F8E82083F8EC2083F8F02083F889
:10036000F42083F8F82083F8FC2083F89C00C1F384
:100370000740090E83F8B00083F8B41083F8AC206E
:100380001A7783F8082193F8942002F0D40242F0FF
:10039000010283F89420704700700440009EFF1F04
:1003A000024B4FF400125A60704700BF00E100E0BA
:1003B000034B4FF40012C3F884215A60704700BF0A
:1003C00000E100E010B5FEF78DF9044618B9FFF71B
:1003D000EFFF204610BD1B2010BD00BF034B4AF2AB
:1003E00002629A814BF280429A8170470020054058
:1003F00081F0004102E000BF83F0004330B54FEAD6
:1004000041044FEA430594EA050F08BF90EA020F42
:100410001FBF54EA000C55EA020C7FEA645C7FEAD5
:10042000655C00F0E2804FEA5454D4EB5555B8BFF8
:100430006D420CDD2C4480EA020281EA030382EA69
:10044000000083EA010180EA020281EA0303362DFB
:1004500088BF30BD11F0004F4FEA01314FF4801CCE
:100460004CEA113102D0404261EB410113F0004FE0
:100470004FEA03334CEA133302D0524263EB430397
:1004800094EA050F00F0A780A4F10104D5F1200E35
:100490000DDB02FA0EFC22FA05F2801841F1000190
:1004A00003FA0EF2801843FA05F359410EE0A5F164
:1004B00020050EF1200E012A03FA0EFC28BF4CF095
:1004C000020C43FA05F3C01851EBE37101F000454B
:1004D00007D54FF0000EDCF1000C7EEB00006EEB58
:1004E0000101B1F5801F1BD3B1F5001F0CD34908E2
:1004F0005FEA30004FEA3C0C04F101044FEA445239
:1005000012F5800F80F09A80BCF1004F08BF5FEABF
:10051000500C50F1000041EB045141EA050130BD9F
:100520005FEA4C0C404141EB010111F4801FA4F142
:100530000104E9D191F0000F04BF01460020B1FA97
:1005400081F308BF2033A3F10B03B3F120020CDACF
:100550000C3208DD02F1140CC2F10C0201FA0CF0AD
:1005600021FA02F10CE002F11402D8BFC2F1200C12
:1005700001FA02F120FA0CFCDCBF41EA0C019040C8
:10058000E41AA2BF01EB0451294330BD6FEA040411
:100590001F3C1CDA0C340EDC04F11404C4F12002FC
:1005A00020FA04F001FA02F340EA030021FA04F30E
:1005B00045EA030130BDC4F10C04C4F1200220FA65
:1005C00002F001FA04F340EA0300294630BD21FAA3
:1005D00004F0294630BD94F0000F83F4801306BF69
:1005E00081F480110134013D4EE77FEA645C18BF5D
:1005F0007FEA655C29D094EA050F08BF90EA020FF4
:1006000005D054EA000C04BF1946104630BD91EAEB
:10061000030F1EBF0021002030BD5FEA545C05D1EE
:100620004000494128BF41F0004130BD14F580042D
:100630003CBF01F5801130BD01F0004545F0FE41A1
:1006400041F470014FF0000030BD7FEA645C1ABFD6
:10065000194610467FEA655C1CBF0B46024650EA0D
:10066000013406BF52EA033591EA030F41F4002139
:1006700030BD00BF90F0000F04BF0021704730B5BF
:100680004FF4806404F132044FF000054FF0000194
:1006900050E700BF90F0000F04BF0021704730B555
:1006A0004FF4806404F1320410F0004548BF40422A
:1006B0004FF000013EE700BF42004FEAE2014FEA7F
:1006C00031014FEA02701FBF12F07F4393F07F4F5A
:1006D00081F06051704792F0000F14BF93F07F4F8C
:1006E000704730B54FF4607401F0004521F00041CF
:1006F00020E700BF50EA010208BF704730B54FF055
:1007000000050AE050EA010208BF704730B511F059
:10071000004502D5404261EB41014FF4806404F191
:1007200032045FEA915C3FF4DCAE4FF003025FEA13
:10073000DC0C18BF03325FEADC0C18BF033202EB9B
:10074000DC02C2F1200300FA03FC20FA02F001FAF5
:1007500003FE40EA0E0021FA02F11444C1E600BF94
:1007600070B54FF0FF0C4CF4E06C1CEA11541DBF47
:100770001CEA135594EA0C0F95EA0C0F00F0DEF812
:100780002C4481EA030621EA4C5123EA4C5350EAF7
:10079000013518BF52EA033541F4801143F4801348
:1007A00038D0A0FB02CE4FF00005E1FB02E506F0D9
:1007B0000042E0FB03E54FF00006E1FB03569CF02E
:1007C000000F18BF4EF0010EA4F1FF04B6F5007F34
:1007D00064F5407404D25FEA4E0E6D4146EB0606A6
:1007E00042EAC62141EA55514FEAC52040EA5E502F
:1007F0004FEACE2EB4F1FD0C88BFBCF5E06F1ED8D9
:10080000BEF1004F08BF5FEA500E50F1000041EB0F
:10081000045170BD06F0004646EA010140EA0200BC
:1008200081EA0301B4EB5C04C2BFD4EB0C0541EADE
:10083000045170BD41F480114FF0000E013C00F3F3
:10084000AB8014F1360FDEBF002001F0004170BD17
:10085000C4F10004203C35DA0C341BDC04F1140430
:10086000C4F1200500FA05F320FA04F001FA05F2BC
:1008700040EA020001F0004221F0004110EBD37089
:1008800021FA04F642EB06015EEA430E08BF20EAB5
:10089000D37070BDC4F10C04C4F1200500FA04F358
:1008A00020FA05F001FA04F240EA020001F00041EA
:1008B00010EBD37041F100015EEA430E08BF20EA5D
:1008C000D37070BDC4F1200500FA05F24EEA020EA5
:1008D00020FA04F301FA05F243EA020321FA04F0D4
:1008E00001F0004121FA04F220EA020000EBD3708B
:1008F0005EEA430E08BF20EAD37070BD94F0000F8B
:100900000FD101F00046400041EB010111F4801FBE
:1009100008BF013CF7D041EA060195F0000F18BF6F
:10092000704703F00046520043EB030313F4801FAB
:1009300008BF013DF7D043EA0603704794EA0C0F65
:100940000CEA135518BF95EA0C0F0CD050EA41067B
:1009500018BF52EA4306D1D181EA030101F00041F8
:100960004FF0000070BD50EA410606BF1046194620
:1009700052EA430619D094EA0C0F02D150EA01362C
:1009800013D195EA0C0F05D152EA03361CBF10466D
:1009900019460AD181EA030101F0004141F0FE410C
:1009A00041F470014FF0000070BD41F0FE4141F490
:1009B000780170BD70B54FF0FF0C4CF4E06C1CEA90
:1009C00011541DBF1CEA135594EA0C0F95EA0C0F45
:1009D00000F0A7F8A4EB050481EA030E52EA033500
:1009E0004FEA013100F088804FEA03334FF0805521
:1009F00045EA131343EA12634FEA022245EA11154E
:100A000045EA10654FEA00260EF000419D4208BFFE
:100A1000964244F1FD0404F5407402D25B084FEAAB
:100A20003202B61A65EB03055B084FEA32024FF457
:100A300080104FF4002CB6EB020E75EB030E22BFB4
:100A4000B61A754640EA0C005B084FEA3202B6EB74
:100A5000020E75EB030E22BFB61A754640EA5C0023
:100A60005B084FEA3202B6EB020E75EB030E22BFB3
:100A7000B61A754640EA9C005B084FEA3202B6EBB4
:100A8000020E75EB030E22BFB61A754640EADC0073
:100A900055EA060E18D04FEA051545EA16754FEAD5
:100AA00006164FEAC30343EA52734FEAC2025FEAF3
:100AB0001C1CC0D111F4801F0BD141EA00014FF082
:100AC00000004FF0004CB6E711F4801F04BF014353
:100AD0000020B4F1FD0C88BFBCF5E06F3FF6AFAE6F
:100AE000B5EB030C04BFB6EB020C5FEA500C50F1FF
:100AF000000041EB045170BD0EF0004E4EEA113182
:100B000014EB5C04C2BFD4EB0C0541EA045170BD88
:100B100041F480114FF0000E013C90E645EA060ECC
:100B20008DE60CEA135594EA0C0F08BF95EA0C0FFA
:100B30003FF43BAF94EA0C0F0AD150EA01347FF442
:100B400034AF95EA0C0F7FF425AF104619462CE719
:100B500095EA0C0F06D152EA03353FF4FDAE10467C
:100B6000194622E750EA410618BF52EA43067FF4CD
:100B7000C5AE50EA41047FF40DAF52EA43057FF45D
:100B8000EBAE12E74FF0FF3C06E000BF4FF0010C68
:100B900002E000BF4FF0010C4DF804CD4FEA410CCC
:100BA0007FEA6C5C4FEA430C18BF7FEA6C5C1BD099
:100BB00001B050EA410C0CBF52EA430C91EA030F1A
:100BC00002BF90EA020F0020704710F1000F91EA77
:100BD000030F58BF994208BF90422CBFD8176FEA45
:100BE000E37040F0010070474FEA410C7FEA6C5C13
:100BF00002D150EA013C07D14FEA430C7FEA6C5C1A
:100C0000D6D152EA033CD3D05DF8040B704700BF45
:100C10008446104662468C461946634600E000BF93
:100C200001B5FFF7B7FF002848BF10F1000F01BD65
:100C30004DF808EDFFF7F4FF0CBF012000205DF830
:100C400008FB00BF4DF808EDFFF7EAFF34BF0120B5
:100C500000205DF808FB00BF4DF808EDFFF7E0FF4E
:100C600094BF012000205DF808FB00BF4DF808ED9F
:100C7000FFF7CEFF94BF012000205DF808FB00BF06
:100C80004DF808EDFFF7C4FF34BF012000205DF8E8
:100C900008FB00BF4FEA410212F5001215D211D530
:100CA0006FF47873B3EB625212D94FEAC12343F069
:100CB000004343EA505311F0004F23FA02F018BFEB
:100CC000404270474FF00000704750EA013005D1B4
:100CD00011F0004008BF6FF0004070474FF0000077
:100CE000704700BF80F0004002E000BF81F000418B
:100CF00042001FBF5FEA410392EA030F7FEA226CC2
:100D00007FEA236C6AD04FEA1262D2EB1363C1BF51
:100D1000D218414048404140B8BF5B42192B88BFC0
:100D2000704710F0004F40F4000020F07F4018BFE3
:100D3000404211F0004F41F4000121F07F4118BF03
:100D4000494292EA030F3FD0A2F1010241FA03FCAB
:100D500010EB0C00C3F1200301FA03F100F0004393
:100D600002D5494260EB4000B0F5000F13D3B0F15B
:100D7000807F06D340084FEA310102F10102FE2ACA
:100D800051D2B1F1004F40EBC25008BF20F001003A
:100D900040EA03007047490040EB000010F4000FE8
:100DA000A2F10102EDD1B0FA80FCACF1080CB2EB7B
:100DB0000C0200FA0CF0AABF00EBC25052421843DA
:100DC000BCBFD0401843704792F0000F81F400017F
:100DD00006BF80F400000132013BB5E74FEA410352
:100DE0007FEA226C18BF7FEA236C21D092EA030FBE
:100DF00004D092F0000F08BF0846704790EA010F38
:100E00001CBF0020704712F07F4F04D1400028BF64
:100E100040F00040704712F100723CBF00F5000046
:100E2000704700F0004343F0FE4040F4000070477C
:100E30007FEA226216BF08467FEA23630146420228
:100E400006BF5FEA412390EA010F40F4800070473B
:100E50004FF0000304E000BF10F0004348BF4042E1
:100E60005FEA000C08BF704743F0964301464FF01D
:100E700000001CE050EA010208BF70474FF0000379
:100E80000AE000BF50EA010208BF704711F00043BA
:100E900002D5404261EB41015FEA010C02BF84468A
:100EA0000146002043F0B64308BFA3F18053A3F5E9
:100EB0000003BCFA8CF2083AA3EBC25310DB01FA30
:100EC00002FC634400FA02FCC2F12002BCF1004FB4
:100ED00020FA02F243EB020008BF20F00100704745
:100EE00002F1200201FA02FCC2F1200250EA4C0099
:100EF00021FA02F243EB020008BF20EADC707047DF
:100F00004FF0FF0C1CEAD0521EBF1CEAD15392EAEC
:100F10000C0F93EA0C0F6FD01A4480EA010C4002C8
:100F200018BF5FEA41211ED04FF0006343EA501022
:100F300043EA5111A0FB01310CF00040B1F5000F64
:100F40003EBF490041EAD3715B0040EA010062F113
:100F50007F02FD2A1DD8B3F1004F40EBC25008BFFD
:100F600020F00100704790F0000F0CF0004C08BF1B
:100F700049024CEA502040EA51207F3AC2BFD2F1E8
:100F8000FF0340EAC250704740F400004FF00003F6
:100F9000013A5DDC12F1190FDCBF00F00040704730
:100FA000C2F10002410021FA02F1C2F1200200FA6E
:100FB00002FC5FEA310040F1000053EA4C0308BF35
:100FC00020EADC70704792F0000F00F0004C02BF86
:100FD000400010F4000F013AF9D040EA0C0093F001
:100FE000000F01F0004C02BF490011F4000F013B5B
:100FF000F9D041EA0C018FE70CEAD15392EA0C0FC9
:1010000018BF93EA0C0F0AD030F0004C18BF31F033
:10101000004CD8D180EA010000F00040704790F009
:10102000000F17BF90F0004F084691F0000F91F0AD
:10103000004F14D092EA0C0F01D142020FD193EA73
:101040000C0F03D14B0218BF084608D180EA0100FB
:1010500000F0004040F0FE4040F40000704740F0D7
:10106000FE4040F4400070474FF0FF0C1CEAD052A5
:101070001EBF1CEAD15392EA0C0F93EA0C0F69D001
:10108000A2EB030280EA010C49024FEA402037D06C
:101090004FF0805343EA111143EA10130CF0004063
:1010A0008B4238BF5B0042F17D024FF4000C8B4253
:1010B00024BF5B1A40EA0C00B3EB510F24BFA3EB33
:1010C000510340EA5C00B3EB910F24BFA3EB910303
:1010D00040EA9C00B3EBD10F24BFA3EBD10340EA5D
:1010E000DC001B0118BF5FEA1C1CE0D1FD2A3FF6A3
:1010F00050AF8B4240EBC25008BF20F00100704758
:101100000CF0004C4CEA50207F32C2BFD2F1FF03FA
:1011100040EAC250704740F400004FF00003013A2B
:1011200037E792F0000F00F0004C02BF400010F4CF
:10113000000F013AF9D040EA0C0093F0000F01F0E3
:10114000004C02BF490011F4000F013BF9D041EA05
:101150000C0195E70CEAD15392EA0C0F08D1420238
:101160007FF47DAF93EA0C0F7FF470AF084676E70B
:1011700093EA0C0F04D14B023FF44CAF08466EE7E4
:1011800030F0004C18BF31F0004CCAD130F00042B2
:101190007FF45CAF31F000437FF43CAF5FE700BF0A
:1011A000FDF737F9002100F004B80C4B5B584350B1
:1011B00004310B480B4B42189A42FFF4F6AF0A4A2F
:1011C00000F003B8002313600432084B9A42FFF486
:1011D000F9AF00F00DF88047704700007819010062
:1011E0000880FF1F6885FF1F0086FF1F00A2FF1FEA
:1011F000264C08B5F7F739F9F7F7A2F9F7F7ECFA43
:10120000F7F700FBF7F704FAF7F7BEFCFBF7C2FEAF
:10121000FBF7E2FDF7F727FEF7F782FBE08CF7F725
:1012200075FC2078F7F704FAE078F7F771FAF7F72A
:101230001FFC28B1F7F71CFC6070F7F719FCA060E1
:10124000F7F77EFCFDF75CF8FCF735FCFCF7C0FD1A
:101250000F4B4FF400725A60FAF7C2FBFAF7ECFF3B
:101260000C4B04225A60FAF7DFFCFBF70BF8FAF795
:10127000E4FFF7F705FCF7F739FC18B1FCF71BFCA6
:10128000FAF7AEFBFDF766F8EDE700BF0C80FF1F35
:1012900080F00F4000F00F40F0B4840743D0541E9C
:1012A000002A3ED0CDB2034603E0621E002C38D0A7
:1012B000144603F8015B9A07F7D1032C2AD9CDB263
:1012C00045EA05250F2C45EA054515D9A4F1100777
:1012D0003F0903F1100606EB07161A461560556024
:1012E0009560D5601032B242F8D104F00F04013796
:1012F000032C03EB07130DD91E462246043A032A9A
:1013000046F8045BFAD8221F22F003020432134489
:1013100004F003042CB1C9B21C4403F8011BA3421E
:10132000FBD1F0BC704714460346C6E7C1F30A5C24
:10133000F8B5ACF2FF33132B06460F4610DC002B3A
:1013400039DBDFF888C04CFA03F303EA010C5CEAEE
:10135000000C1AD107F000416046C2E90067F8BDF1
:10136000332B1CDC4FF0FF33ACF2134C23FA0CFC94
:101370001CEA000319D020EA0C060F46C2E90067F8
:101380000B463246FFF738F8F8BD21EA030700267E
:10139000C2E900673B463246FFF72EF8F8BD07F07A
:1013A00000410020C2E90067F8BD07F0004118467F
:1013B000C2E90067F8BD07F00041002004460D4671
:1013C00030463946C2E90045F8BD00BFFFFF0F00B7
:1013D000024B13B1024800F005B87047000000004E
:1013E000F1130100014600200246034600F018B840
:1013F00038B5094D094C641BA41018BF05EB8405D2
:1014000005D0013C55F8043D9847002CF9D1BDE8C2
:10141000384000F0A5BA00BF741901007819010026
:10142000F0B5274C2668D6F8484185B00746002C11
:1014300041D065681F2D1EDD224818B94FF0FF30DE
:1014400005B0F0BD4FF4C870039102920193AFF361
:1014500000800399029A019B04460028EED0D6F83A
:1014600048512560002060600546C6F84841C4F830
:101470008801C4F88C013FB9AB1C002001356560C0
:1014800044F8231005B0F0BD04EB85004FF0010CCB
:10149000C0F88820D4F888610CFA05F21643022FB0
:1014A000C4F88861C0F80831E6D1D4F88C311A4309
:1014B000C4F88C21E0E706F5A674C6F84841B8E701
:1014C00050190100000000002DE9F84FC1F30A5740
:1014D000A7F2FF36132E02460B4604460D468946F8
:1014E0008A46804622DC002E54DB3D4F374107EA16
:1014F000010C5CEA000C1ED037A3D3E90023FEF7F1
:101500007DFF00220023FFF7BBFB58B1002D05DD56
:101510004FF4801A4AFA06F606EB050A2AEA07098A
:101520004FF0000840464946BDE8F88F332E06DDEF
:10153000B6F5806F43D010461946BDE8F88FA7F284
:10154000134C4FF0FF3B2BFA0CFB1BEA000FF2D0C1
:1015500021A3D3E90023FEF751FF00220023FFF768
:101560008FFB0028DED0002D0DDD142E09D0C7F52D
:10157000866703374FF0010808FA07F818EB0408EC
:1015800001D305F1010A28EA0B08D1464046494635
:10159000BDE8F88F10A3D3E90023FEF72FFF002248
:1015A0000023FFF76DFB0028BCD0002D0DDB55EAB2
:1015B000040808D0DFF82C904FF00008B2E7FEF7DF
:1015C0001DFFBDE8F88FC146ACE74FF000084FF0B3
:1015D0000049A7E7AFF300809C7500883CE4377EA4
:1015E000FFFF0F000000F03F2DE9F84FC1F30A574D
:1015F000A7F2FF36132E02460B4604460D468946D7
:101600008A4680461CDC002E40DB3D4F374107EA0E
:10161000010C5CEA000C18D037A3D3E90023FEF7D5
:10162000EDFE00220023FFF72BFB28B1002D42DB4B
:101630002AEA07094FF0000840464946BDE8F88FFE
:10164000332E06DDB6F5806F31D010461946BDE861
:10165000F88FA7F2134C4FF0FF3B2BFA0CFB1BEA61
:10166000000FF2D024A3D3E90023FEF7C7FE002227
:101670000023FFF705FB0028DED0002D22DB28EA3F
:101680000B08D14640464946BDE8F88F1AA3D3E976
:101690000023FEF7B3FE00220023FFF7F1FA002833
:1016A000CAD0002D1CDB4FF00008C146C4E7FEF78E
:1016B000A5FEBDE8F88F4FF4801A4AFA06F606EB4D
:1016C000050AB5E7142E14D0C7F586670123033742
:1016D00003FA07F717EB040828BF05EB030ACEE768
:1016E00025F00042074B224318BF99464FF00008EF
:1016F000A2E705F1010AC2E79C7500883CE4377E49
:10170000FFFF0F000000F0BF802500004038000000
:10171000004B0000807000000096000000E1000017
:10172000002C010000C201000084030090D00300DF
:1017300020A1070040420F0050C3000088130000A2
:10174000018008080000000000000000C800000040
:101750000100C80000800000000000000000000040
:101760000000000000000000000000000000000079
:10177000000000000000000001000200040008005A
:101780001000200001010100010000000000000025
:101790000000000000010000000000000001000047
:1017A0000000000001010100000000000000000036
:1017B0000001000000000000010101000101000122
:1017C0000100000001010100000000000000000015
:1017D0000001000000000000010101000101000102
:1017E00001000000000000000000000000000101F6
:1017F00001000001000000000000000000000101E5
:101800000100000108000000040000005780FF1FD5
:101810000400000009040000701801008018010095
:1018200000000000000000000000000000000000B8
:101830002E81FF1FEB80FF1F000000000000000052
:101840000000000000000000000000000000120086
:10185000430000000000000000000000030102013E
:10186000100002020010000303011000000100003C
:101870005780FF1FB180FF1F8B80FF1F6980FF1FF4
:10188000043A26226501010069EA0000FDEA000031
:101890006DE800008DFC00008DFC00008DFC000058
:1018A0008DFC00008DFC00008DFC00008DFC000014
:1018B0008DFC00008DFC00008DFC00008DFC000004
:1018C0008DFC0000FFED000099ED0000F5ED00003B
:1018D000C1ED000099ED00008DFC000081ED0000DD
:1018E0006DEE000029FF0000F5FF00000000000081
:1018F000F5FF000000000000E9FE000011FF0000FD
:101900000000000055FE000085FE0000EB00010015
:10191000C900010029FE00000101000101000000D2
:1019200000010100000000000101010101000000B0
:1019300001010001010001000001000001000000A0
:1019400036323131563130330000000043000000A0
:101950004081FF1FF8B500BFF8BC08BC9E46704729
:0C196000F8B500BFF8BC08BC9E467047FC
:08196C00D113010035840000D5
:0419740011840000DA
:1019780040190100000102000008000001000000F9
:10198800020000000000000000000000000000004D
:10199800000000000000000000000000000000003F
:1019A800000000000000000000000000000000002F
:1019B80000000000A1200000000002000000FF0459
:1019C80003090400C2010000000800000000000034
:1019D80000220342004100440020005300540052FA
:1019E8000049004E004700200049004E00440045D1
:1019F80000580026035300740065007000700065ED
:101A080000720020004D006F0074006F007200200B
:101A18000044006500760020003A03540052004953
:101A2800004E0041004D004900430020004D006F6A
:101A380000740069006F006E00200043006F006EA4
:101A480000740072006F006C00200020002000204D
:101A580000200009024300020100C032090400000E
:101A680001020200000524001001052401010104FF
:101A780024020605240600010705830310000A094D
:101A8800040100020A000000070581021000000797
:101A980005020210000012010002020000103C2A98
:101AA8000001020001020001000000002C84FF1F59
:101AB8009484FF1FFC84FF1F00000000000000004A
:101AC800000000000000000000000000000000000E
:101AD8000000000000000000000000004C19010098
:101AE80000000000000000000000000000000000EE
:101AF80000000000000000000000000000000000DE
:101B080000000000000000000000000000000000CD
:101B180000000000000000000000000000000000BD
:101B280000000000000000000000000000000000AD
:101B3800000000000000000000000000000000009D
:101B4800000000000000000000000000000000008D
:101B580001000000000000000E33CDAB34126DE62A
:101B6800ECDE05000B000000000000000000000093
:101B7800000000000000000000000000000000005D
:101B8800000000000000000000000000000000004D
:101B9800000000000000000000000000000000003D
:101BA800000000000000000000000000000000002D
:101ED800781901000880FF1F60050000000000005D
:081EE8000000000000000000F2
:020000020000FC
:020000041FFFDC
:04800000000000007C
:04000003100011A137
:00000001FF
